******************************************************************************
               TMS320C6x Linker Unix v7.4.18                   
******************************************************************************
>> Linked Thu Sep 21 14:33:42 2017

OUTPUT FILE NAME:   <Test_bios.out>
ENTRY POINT SYMBOL: "_c_int00"  address: 80009680


MEMORY CONFIGURATION

         name            origin    length      used     unused   attr    fill
----------------------  --------  ---------  --------  --------  ----  --------
  L2SRAM                00800000   00040000  00000000  00040000  RW X
  OCMC_RAM1             40300000   00080000  00000000  00080000  RW X
  OCMC_RAM2             40400000   00100000  00000000  00100000  RW X
  OCMC_RAM3             40500000   00100000  00000000  00100000  RW X
  EXT_RAM               80000000   80000000  00013de6  7ffec21a  RWIX


SEGMENT ALLOCATION MAP

run origin  load origin   length   init length attrs members
----------  ----------- ---------- ----------- ----- -------
80000000    80000000    0000f40a   0000f40a    r-x
  80000000    80000000    0000c680   0000c680    r-x .text
  8000c680    8000c680    00002d8a   00002d8a    r-- .const
8000f410    8000f410    00003c08   00000000    rw-
  8000f410    8000f410    00002000   00000000    rw- .stack
  80011410    80011410    00001c08   00000000    rw- .far
80013018    80013018    00000644   00000644    rw-
  80013018    80013018    00000644   00000644    rw- .fardata
80013660    80013660    00000120   00000000    rw-
  80013660    80013660    00000120   00000000    rw- .cio
80013800    80013800    00000670   00000670    r-x
  80013800    80013800    00000200   00000200    r-x .vecs
  80013a00    80013a00    00000470   00000470    r-- .cinit


SECTION ALLOCATION MAP

 output                                  attributes/
section   page    origin      length       input sections
--------  ----  ----------  ----------   ----------------
.init_array 
*          0    80000000    00000000     UNINITIALIZED

xdc.meta   0    80000000    000000e8     COPY SECTION
                  80000000    000000e8     app_pe66.oe66 (xdc.meta)

.text      0    80000000    0000c680     
                  80000000    00000880     ti.targets.rts6000.ae66 : System.oe66 (.text:xdc_runtime_System_doPrint__I)
                  80000880    00000780     sysbios.ae66 : BIOS.obj (.text:ti_sysbios_family_c64p_Exception_handler__I)
                  80001000    00000780                  : BIOS.obj (.text:ti_sysbios_knl_Semaphore_pend__E)
                  80001780    000005e0                  : BIOS.obj (.text:ti_sysbios_heaps_HeapMem_allocUnprotected__E)
                  80001d60    000005a0                  : BIOS.obj (.text:ti_sysbios_heaps_HeapMem_freeUnprotected__E)
                  80002300    000004a0                  : BIOS.obj (.text:ti_sysbios_knl_Task_Instance_finalize__E)
                  800027a0    00000480                  : BIOS.obj (.text:ti_sysbios_knl_Task_sleep__E)
                  80002c20    000003a0                  : BIOS.obj (.text:ti_sysbios_timers_dmtimer_Timer_checkFreq__I)
                  80002fc0    00000380                  : BIOS.obj (.text:ti_sysbios_knl_Task_Instance_init__E)
                  80003340    00000360                  : BIOS.obj (.text:ti_sysbios_timers_dmtimer_Timer_deviceConfig__I)
                  800036a0    000002e0                  : BIOS.obj (.text:ti_sysbios_heaps_HeapMem_Instance_init__E)
                  80003980    000002e0                  : BIOS.obj (.text:ti_sysbios_knl_Task_Module_startup__E)
                  80003c60    000002a0                  : BIOS.obj (.text:ti_sysbios_knl_Clock_workFunc__E)
                  80003f00    00000280                  : BIOS.obj (.text:ti_sysbios_knl_Semaphore_post__E)
                  80004180    00000280     ti.targets.rts6000.ae66 : LoggerBuf.oe66 (.text:xdc_runtime_LoggerBuf_write8__E)
                  80004400    00000260     sysbios.ae66 : BIOS.obj (.text:ti_sysbios_family_c64p_Hwi_dispatchCore__I)
                  80004660    00000260     app_pe66.oe66 (.text:xdc_runtime_System_printfExtend__I)
                  800048c0    00000240     rts6600_elf.lib : imath64.obj (.text:__c6xabi_divull)
                  80004b00    00000240     sysbios.ae66 : BIOS.obj (.text:ti_sysbios_family_c64p_Exception_internalHandler__I)
                  80004d40    00000240                  : BIOS.obj (.text:ti_sysbios_timers_dmtimer_Timer_setPeriodMicroSecs__E)
                  80004f80    00000220                  : BIOS.obj (.text:ti_sysbios_knl_Swi_run__I)
                  800051a0    00000220     ti.targets.rts6000.ae66 : Core-mem.oe66 (.text:xdc_runtime_Core_createObject__I)
                  800053c0    00000200     sysbios.ae66 : c64p_Hwi_disp_always.obj (.text:_ti_sysbios_family_c64p_Hwi_dispatchAlways)
                  800055c0    000001e0     ti.targets.rts6000.ae66 : Error.oe66 (.text:xdc_runtime_Error_policyDefault__E)
                  800057a0    000001e0                             : Startup.oe66 (.text:xdc_runtime_Startup_startMods__I)
                  80005980    000001c0     sysbios.ae66 : BIOS.obj (.text:ti_sysbios_family_c66_Cache_block__I)
                  80005b40    000001c0                  : BIOS.obj (.text:ti_sysbios_knl_Task_checkStacks__E)
                  80005d00    000001c0                  : BIOS.obj (.text:ti_sysbios_knl_Task_exit__E)
                  80005ec0    000001c0     ti.targets.rts6000.ae66 : LoggerBuf.oe66 (.text:xdc_runtime_LoggerBuf_write4__E)
                  80006080    000001c0                             : Text.oe66 (.text:xdc_runtime_Text_putSite__E)
                  80006240    000001a0     sysbios.ae66 : BIOS.obj (.text:ti_sysbios_gates_GateMutex_enter__E)
                  800063e0    000001a0                  : BIOS.obj (.text:ti_sysbios_knl_Task_schedule__I)
                  80006580    00000180     rts6600_elf.lib : copy_decompress_rle.obj (.text:__TI_decompress_rle_core)
                  80006700    00000180     sysbios.ae66 : c64p_Exception_asm.obj (.text)
                  80006880    00000180                  : BIOS.obj (.text:ti_sysbios_knl_Task_startCore__E)
                  80006a00    00000180     ti.targets.rts6000.ae66 : Core-smem.oe66 (.text:xdc_runtime_Core_constructObject__I)
                  80006b80    00000160     sysbios.ae66 : BIOS.obj (.text:ti_sysbios_family_c66_Cache_getL2InitSize__I)
                  80006ce0    00000160                  : BIOS.obj (.text:ti_sysbios_knl_Swi_post__E)
                  80006e40    00000160                  : BIOS.obj (.text:ti_sysbios_timers_dmtimer_Timer_start__E)
                  80006fa0    00000140     boot.ae66 : autoinit.oe66 (.text:_auto_init_elf)
                  800070e0    00000140     sysbios.ae66 : BIOS.obj (.text:ti_sysbios_family_c64p_Hwi_Module_startup__E)
                  80007220    00000140                  : BIOS.obj (.text:ti_sysbios_family_c66_Cache_startup__I)
                  80007360    00000140                  : BIOS.obj (.text:ti_sysbios_knl_Semaphore_Instance_init__E)
                  800074a0    00000140                  : BIOS.obj (.text:ti_sysbios_knl_Task_blockI__E)
                  800075e0    00000140                  : BIOS.obj (.text:ti_sysbios_knl_Task_postInit__I)
                  80007720    00000120                  : BIOS.obj (.text:ti_sysbios_family_c66_Cache_getL1DInitSize__I)
                  80007840    00000120                  : BIOS.obj (.text:ti_sysbios_family_c66_Cache_getL1PInitSize__I)
                  80007960    00000120                  : BIOS.obj (.text:ti_sysbios_timers_dmtimer_Timer_Module_startup__E)
                  80007a80    00000120                  : BIOS.obj (.text:ti_sysbios_timers_dmtimer_Timer_initDevice__I)
                  80007ba0    00000120     ti.targets.rts6000.ae66 : Core-mem.oe66 (.text:xdc_runtime_Core_deleteObject__I)
                  80007cc0    00000120                             : LoggerBuf.oe66 (.text:xdc_runtime_LoggerBuf_setFilterLevel__E)
                  80007de0    00000120                             : Text.oe66 (.text:xdc_runtime_Text_putLab__E)
                  80007f00    00000120                             : Text.oe66 (.text:xdc_runtime_Text_putMod__E)
                  80008020    00000100     sysbios.ae66 : BIOS.obj (.text:ti_sysbios_knl_Swi_restoreHwi__E)
                  80008120    00000100                  : BIOS.obj (.text:ti_sysbios_knl_Swi_schedule__I)
                  80008220    00000100                  : BIOS.obj (.text:ti_sysbios_knl_Task_unblockI__E)
                  80008320    00000100     ti.targets.rts6000.ae66 : LoggerBuf.oe66 (.text:xdc_runtime_LoggerBuf_getFilterLevel__E)
                  80008420    00000100                             : Startup.oe66 (.text:xdc_runtime_Startup_exec__E)
                  80008520    000000e0     rts6600_elf.lib : copy_zero_init.obj (.text:decompress:ZI:__TI_zero_init)
                  80008600    000000e0                     : memset.obj (.text:memset)
                  800086e0    000000e0     sysbios.ae66 : BIOS.obj (.text:ti_sysbios_knl_Swi_runLoop__I)
                  800087c0    000000e0                  : BIOS.obj (.text:ti_sysbios_knl_Swi_startup__E)
                  800088a0    000000e0                  : BIOS.obj (.text:ti_sysbios_timers_dmtimer_Timer_startup__E)
                  80008980    000000e0     ti.targets.rts6000.ae66 : Error.oe66 (.text:xdc_runtime_Error_print__E)
                  80008a60    000000e0                             : Memory.oe66 (.text:xdc_runtime_Memory_alloc__E)
                  80008b40    000000e0                             : Text.oe66 (.text:xdc_runtime_Text_visitRope2__I)
                  80008c20    000000c0     rts6600_elf.lib : trgdrv.obj (.text:HOSTwrite)
                  80008ce0    000000c0                     : divu.obj (.text:__divu)
                  80008da0    000000c0                     : exit.obj (.text:exit)
                  80008e60    000000c0     main.obj (.text)
                  80008f20    000000c0     sysbios.ae66 : BIOS.obj (.text:ti_sysbios_heaps_HeapMem_alloc__E)
                  80008fe0    000000c0                  : BIOS.obj (.text:ti_sysbios_heaps_HeapMem_getStats__E)
                  800090a0    000000c0                  : BIOS.obj (.text:ti_sysbios_knl_Clock_logTick__E)
                  80009160    000000c0                  : BIOS.obj (.text:ti_sysbios_knl_Task_allBlockedFunction__I)
                  80009220    000000c0     app_pe66.oe66 (.text:ti_sysbios_knl_Task_create)
                  800092e0    000000c0     sysbios.ae66 : BIOS.obj (.text:ti_sysbios_timers_dmtimer_Timer_stop__E)
                  800093a0    000000c0     rts6600_elf.lib : tls.obj (.text:tls:init:__TI_tls_init)
                  80009460    000000c0     app_pe66.oe66 (.text:xdc_runtime_LoggerBuf_Object__create__S)
                  80009520    000000c0     ti.targets.rts6000.ae66 : System.oe66 (.text:xdc_runtime_System_formatNum__I)
                  800095e0    000000a0     rts6600_elf.lib : remu.obj (.text:__remu)
                  80009680    000000a0     boot.ae66 : boot.oe66 (.text:_c_int00)
                  80009720    000000a0     rts6600_elf.lib : memcpy64.obj (.text:memcpy)
                  800097c0    000000a0     sysbios.ae66 : BIOS.obj (.text:ti_sysbios_family_c64p_Exception_Module_startup__E)
                  80009860    000000a0                  : BIOS.obj (.text:ti_sysbios_heaps_HeapMem_init__I)
                  80009900    000000a0     ti.targets.rts6000.ae66 : Assert.oe66 (.text:xdc_runtime_Assert_raise__I)
                  800099a0    000000a0                             : Error.oe66 (.text:xdc_runtime_Error_setX__E)
                  80009a40    000000a0                             : SysMin.oe66 (.text:xdc_runtime_SysMin_abort__E)
                  80009ae0    000000a0                             : SysMin.oe66 (.text:xdc_runtime_SysMin_flush__E)
                  80009b80    000000a0                             : SysMin.oe66 (.text:xdc_runtime_SysMin_putch__E)
                  80009c20    000000a0                             : Text.oe66 (.text:xdc_runtime_Text_xprintf__I)
                  80009cc0    00000080     rts6600_elf.lib : llshift.obj (.text:__c6xabi_llshl)
                  80009d40    00000080     sysbios.ae66 : c62_TaskSupport_asm.obj (.text:_ti_sysbios_family_c62_TaskSupport_swap__E)
                  80009dc0    00000080     rts6600_elf.lib : trgmsg.obj (.text:readmsg)
                  80009e40    00000080     sysbios.ae66 : BIOS.obj (.text:ti_sysbios_family_c64p_Hwi_dispatchC__I)
                  80009ec0    00000080                  : BIOS.obj (.text:ti_sysbios_family_c64p_Hwi_getStackInfo__E)
                  80009f40    00000080                  : BIOS.obj (.text:ti_sysbios_hal_Hwi_checkStack)
                  80009fc0    00000080                  : BIOS.obj (.text:ti_sysbios_hal_Hwi_initStack)
                  8000a040    00000080                  : BIOS.obj (.text:ti_sysbios_knl_Idle_run__E)
                  8000a0c0    00000080                  : BIOS.obj (.text:ti_sysbios_knl_Task_restore__E)
                  8000a140    00000080     ti.targets.rts6000.ae66 : Core-label.oe66 (.text:xdc_runtime_Core_assignLabel__I)
                  8000a1c0    00000080                             : Core-params.oe66 (.text:xdc_runtime_Core_assignParams__I)
                  8000a240    00000080                             : LoggerBuf.oe66 (.text:xdc_runtime_LoggerBuf_Instance_init__E)
                  8000a2c0    00000080                             : LoggerBuf.oe66 (.text:xdc_runtime_LoggerBuf_Module_startup__E)
                  8000a340    00000080                             : LoggerBuf.oe66 (.text:xdc_runtime_LoggerBuf_filterOutEvent__I)
                  8000a3c0    00000080                             : System.oe66 (.text:xdc_runtime_System_atexit__E)
                  8000a440    00000080                             : System.oe66 (.text:xdc_runtime_System_processAtExit__E)
                  8000a4c0    00000080                             : System.oe66 (.text:xdc_runtime_System_putchar__I)
                  8000a540    00000080                             : Text.oe66 (.text:xdc_runtime_Text_printVisFxn__I)
                  8000a5c0    00000060     rts6600_elf.lib : llshift.obj (.text:__c6xabi_llshru)
                  8000a620    00000060                     : imath64.obj (.text:_subcull)
                  8000a680    00000060     sysbios.ae66 : c64p_Hwi_asm_switch.obj (.text:_ti_sysbios_family_c64p_Hwi_switchAndDispatch__I)
                  8000a6e0    00000060                  : c64p_Hwi_asm_switch.obj (.text:_ti_sysbios_family_xxx_Hwi_switchAndRunFunc)
                  8000a740    00000060     app_pe66.oe66 (.text:ti_sysbios_BIOS_atExitFunc__I)
                  8000a7a0    00000060     app_pe66.oe66 (.text:ti_sysbios_BIOS_errorRaiseHook__I)
                  8000a800    00000060     app_pe66.oe66 (.text:ti_sysbios_BIOS_registerRTSLock__I)
                  8000a860    00000060     app_pe66.oe66 (.text:ti_sysbios_BIOS_removeRTSLock__I)
                  8000a8c0    00000060     app_pe66.oe66 (.text:ti_sysbios_BIOS_rtsUnlock__I)
                  8000a920    00000060     app_pe66.oe66 (.text:ti_sysbios_BIOS_startFunc__I)
                  8000a980    00000060     sysbios.ae66 : BIOS.obj (.text:ti_sysbios_family_c62_TaskSupport_start__E)
                  8000a9e0    00000060                  : BIOS.obj (.text:ti_sysbios_family_c66_Cache_Module_startup__E)
                  8000aa40    00000060     app_pe66.oe66 (.text:ti_sysbios_gates_GateHwi_Object__create__S)
                  8000aaa0    00000060     app_pe66.oe66 (.text:ti_sysbios_gates_GateMutex_Object__create__S)
                  8000ab00    00000060     app_pe66.oe66 (.text:ti_sysbios_heaps_HeapMem_Object__create__S)
                  8000ab60    00000060     sysbios.ae66 : BIOS.obj (.text:ti_sysbios_heaps_HeapMem_free__E)
                  8000abc0    00000060                  : BIOS.obj (.text:ti_sysbios_knl_Clock_Module_startup__E)
                  8000ac20    00000060     app_pe66.oe66 (.text:ti_sysbios_knl_Clock_doTick__I)
                  8000ac80    00000060     app_pe66.oe66 (.text:ti_sysbios_knl_Queue_construct)
                  8000ace0    00000060     app_pe66.oe66 (.text:ti_sysbios_knl_Semaphore_construct)
                  8000ad40    00000060     sysbios.ae66 : BIOS.obj (.text:ti_sysbios_knl_Semaphore_pendTimeout__I)
                  8000ada0    00000060                  : BIOS.obj (.text:ti_sysbios_knl_Swi_Module_startup__E)
                  8000ae00    00000060                  : BIOS.obj (.text:ti_sysbios_knl_Task_enter__I)
                  8000ae60    00000060                  : BIOS.obj (.text:ti_sysbios_knl_Task_processVitalTaskFlag__I)
                  8000aec0    00000060                  : BIOS.obj (.text:ti_sysbios_timers_dmtimer_Timer_stub__E)
                  8000af20    00000060     rts6600_elf.lib : trgmsg.obj (.text:writemsg)
                  8000af80    00000060     ti.targets.rts6000.ae66 : Memory.oe66 (.text:xdc_runtime_Memory_valloc__E)
                  8000afe0    00000060                             : SysMin.oe66 (.text:xdc_runtime_SysMin_Module_startup__E)
                  8000b040    00000060                             : SysMin.oe66 (.text:xdc_runtime_SysMin_exit__E)
                  8000b0a0    00000060     app_pe66.oe66 (.text:xdc_runtime_SysMin_output__I)
                  8000b100    00000060     ti.targets.rts6000.ae66 : System.oe66 (.text:xdc_runtime_System_avprintf__E)
                  8000b160    00000060                             : System.oe66 (.text:xdc_runtime_System_vprintf__E)
                  8000b1c0    00000060                             : Text.oe66 (.text:xdc_runtime_Text_cordText__E)
                  8000b220    00000040     rts6600_elf.lib : strasg.obj (.text:__strasgi_64plus)
                  8000b260    00000040                     : args_main.obj (.text:_args_main)
                  8000b2a0    00000040     sysbios.ae66 : c62_TaskSupport_asm.obj (.text:_ti_sysbios_family_c62_TaskSupport_buildTaskStack)
                  8000b2e0    00000040     app_pe66.oe66 (.text:ti_sysbios_BIOS_exitFunc__I)
                  8000b320    00000040     app_pe66.oe66 (.text:ti_sysbios_BIOS_rtsLock__I)
                  8000b360    00000040     app_pe66.oe66 (.text:ti_sysbios_family_c64p_Hwi_Module__startupDone__F)
                  8000b3a0    00000040     sysbios.ae66 : BIOS.obj (.text:ti_sysbios_family_c64p_Hwi_disableInterrupt__E)
                  8000b3e0    00000040                  : BIOS.obj (.text:ti_sysbios_family_c64p_Hwi_enableInterrupt__E)
                  8000b420    00000040     app_pe66.oe66 (.text:ti_sysbios_family_shared_vayu_TimerSupport_Module__startupDone__F)
                  8000b460    00000040     app_pe66.oe66 (.text:ti_sysbios_gates_GateHwi_Handle__label__S)
                  8000b4a0    00000040     app_pe66.oe66 (.text:ti_sysbios_gates_GateHwi_Object__delete__S)
                  8000b4e0    00000040     app_pe66.oe66 (.text:ti_sysbios_gates_GateMutex_Handle__label__S)
                  8000b520    00000040     sysbios.ae66 : BIOS.obj (.text:ti_sysbios_gates_GateMutex_Instance_init__E)
                  8000b560    00000040     app_pe66.oe66 (.text:ti_sysbios_gates_GateMutex_Object__delete__S)
                  8000b5a0    00000040     sysbios.ae66 : BIOS.obj (.text:ti_sysbios_gates_GateMutex_leave__E)
                  8000b5e0    00000040     app_pe66.oe66 (.text:ti_sysbios_heaps_HeapMem_Handle__label__S)
                  8000b620    00000040     app_pe66.oe66 (.text:ti_sysbios_heaps_HeapMem_Object__delete__S)
                  8000b660    00000040     app_pe66.oe66 (.text:ti_sysbios_heaps_HeapMem_Object__get__S)
                  8000b6a0    00000040     app_pe66.oe66 (.text:ti_sysbios_knl_Queue_Object__destruct__S)
                  8000b6e0    00000040     app_pe66.oe66 (.text:ti_sysbios_knl_Semaphore_Object__destruct__S)
                  8000b720    00000040     app_pe66.oe66 (.text:ti_sysbios_knl_Swi_Object__get__S)
                  8000b760    00000040     app_pe66.oe66 (.text:ti_sysbios_knl_Task_Object__get__S)
                  8000b7a0    00000040     sysbios.ae66 : BIOS.obj (.text:ti_sysbios_knl_Task_sleepTimeout__I)
                  8000b7e0    00000040     app_pe66.oe66 (.text:ti_sysbios_timers_dmtimer_Timer_Module__startupDone__F)
                  8000b820    00000040     ti.targets.rts6000.ae66 : Error.oe66 (.text:xdc_runtime_Error_check__E)
                  8000b860    00000040                             : Error.oe66 (.text:xdc_runtime_Error_init__E)
                  8000b8a0    00000040     app_pe66.oe66 (.text:xdc_runtime_LoggerBuf_Handle__label__S)
                  8000b8e0    00000040     ti.targets.rts6000.ae66 : LoggerBuf.oe66 (.text:xdc_runtime_LoggerBuf_Instance_finalize__E)
                  8000b920    00000040     app_pe66.oe66 (.text:xdc_runtime_LoggerBuf_Object__delete__S)
                  8000b960    00000040     app_pe66.oe66 (.text:xdc_runtime_LoggerBuf_Object__get__S)
                  8000b9a0    00000040     ti.targets.rts6000.ae66 : LoggerBuf.oe66 (.text:xdc_runtime_LoggerBuf_reset__E)
                  8000b9e0    00000040                             : LoggerBuf.oe66 (.text:xdc_runtime_LoggerBuf_write0__E)
                  8000ba20    00000040                             : Memory.oe66 (.text:xdc_runtime_Memory_free__E)
                  8000ba60    00000040                             : Registry.oe66 (.text:xdc_runtime_Registry_findById__E)
                  8000baa0    00000040                             : System.oe66 (.text:xdc_runtime_System_abort__E)
                  8000bae0    00000040     app_pe66.oe66 (.text:xdc_runtime_System_aprintf__E)
                  8000bb20    00000040     ti.targets.rts6000.ae66 : System.oe66 (.text:xdc_runtime_System_exit__E)
                  8000bb60    00000040     app_pe66.oe66 (.text:xdc_runtime_System_printf__E)
                  8000bba0    00000040     ti.targets.rts6000.ae66 : Text.oe66 (.text:xdc_runtime_Text_ropeText__E)
                  8000bbe0    00000020                             : LoggerBuf.oe66 (.text:LoggerBuf_instanceStartup)
                  8000bc00    00000020                             : xdc_noinit.oe66 (.text:__xdc__init)
                  8000bc20    00000020     rts6600_elf.lib : _lock.obj (.text:_nop)
                  8000bc40    00000020                     : _lock.obj (.text:_register_lock)
                  8000bc60    00000020                     : _data_synch.obj (.text:_register_synch_api)
                  8000bc80    00000020                     : _lock.obj (.text:_register_unlock)
                  8000bca0    00000020     sysbios.ae66 : c62_TaskSupport_asm.obj (.text:_ti_sysbios_family_c62_TaskSupport_glue)
                  8000bcc0    00000020     rts6600_elf.lib : exit.obj (.text:abort)
                  8000bce0    00000020                     : copy_decompress_none.obj (.text:decompress:none:__TI_decompress_none)
                  8000bd00    00000020                     : copy_decompress_rle.obj (.text:decompress:rle24:__TI_decompress_rle24)
                  8000bd20    00000020     app_pe66.oe66 (.text:ti_sysbios_BIOS_RtsGateProxy_enter__E)
                  8000bd40    00000020     app_pe66.oe66 (.text:ti_sysbios_BIOS_RtsGateProxy_leave__E)
                  8000bd60    00000020     sysbios.ae66 : BIOS.obj (.text:ti_sysbios_BIOS_exit__E)
                  8000bd80    00000020                  : BIOS.obj (.text:ti_sysbios_BIOS_getCpuFreq__E)
                  8000bda0    00000020                  : BIOS.obj (.text:ti_sysbios_BIOS_linkedWithIncorrectBootLibrary__E)
                  8000bdc0    00000020     app_pe66.oe66 (.text:ti_sysbios_BIOS_nullFunc__I)
                  8000bde0    00000020     sysbios.ae66 : BIOS.obj (.text:ti_sysbios_BIOS_setThreadType__E)
                  8000be00    00000020                  : BIOS.obj (.text:ti_sysbios_BIOS_start__E)
                  8000be20    00000020     app_pe66.oe66 (.text:ti_sysbios_family_c62_TaskSupport_Module__startupDone__S)
                  8000be40    00000020     sysbios.ae66 : BIOS.obj (.text:ti_sysbios_family_c62_TaskSupport_checkStack__E)
                  8000be60    00000020                  : BIOS.obj (.text:ti_sysbios_family_c62_TaskSupport_getStackAlignment__E)
                  8000be80    00000020                  : BIOS.obj (.text:ti_sysbios_family_c64p_Hwi_clearInterrupt__E)
                  8000bea0    00000020                  : BIOS.obj (.text:ti_sysbios_family_c64p_Hwi_startup__E)
                  8000bec0    00000020                  : BIOS.obj (.text:ti_sysbios_family_c64p_Hwi_switchFromBootStack__E)
                  8000bee0    00000020                  : BIOS.obj (.text:ti_sysbios_family_c64p_TimestampProvider_Module_startup__E)
                  8000bf00    00000020                  : BIOS.obj (.text:ti_sysbios_family_c64p_TimestampProvider_get32__E)
                  8000bf20    00000020                  : BIOS.obj (.text:ti_sysbios_family_c64p_TimestampProvider_get64__E)
                  8000bf40    00000020                  : BIOS.obj (.text:ti_sysbios_family_c66_Cache_RTSSynchInv__I)
                  8000bf60    00000020                  : BIOS.obj (.text:ti_sysbios_family_c66_Cache_RTSSynchWbInv__I)
                  8000bf80    00000020                  : BIOS.obj (.text:ti_sysbios_family_c66_Cache_RTSSynchWb__I)
                  8000bfa0    00000020                  : BIOS.obj (.text:ti_sysbios_family_c66_Cache_wait__E)
                  8000bfc0    00000020                  : BIOS.obj (.text:ti_sysbios_family_shared_vayu_TimerSupport_Module_startup__E)
                  8000bfe0    00000020                  : BIOS.obj (.text:ti_sysbios_family_shared_vayu_TimerSupport_enable__E)
                  8000c000    00000020                  : BIOS.obj (.text:ti_sysbios_gates_GateHwi_Instance_init__E)
                  8000c020    00000020                  : BIOS.obj (.text:ti_sysbios_gates_GateHwi_enter__E)
                  8000c040    00000020                  : BIOS.obj (.text:ti_sysbios_gates_GateHwi_leave__E)
                  8000c060    00000020                  : BIOS.obj (.text:ti_sysbios_gates_GateHwi_query__E)
                  8000c080    00000020                  : BIOS.obj (.text:ti_sysbios_gates_GateMutex_Instance_finalize__E)
                  8000c0a0    00000020                  : BIOS.obj (.text:ti_sysbios_gates_GateMutex_query__E)
                  8000c0c0    00000020     app_pe66.oe66 (.text:ti_sysbios_hal_Hwi_HwiProxy_Module__startupDone__S)
                  8000c0e0    00000020     sysbios.ae66 : BIOS.obj (.text:ti_sysbios_hal_Hwi_Module_startup__E)
                  8000c100    00000020     app_pe66.oe66 (.text:ti_sysbios_heaps_HeapMem_Module_GateProxy_enter__E)
                  8000c120    00000020     app_pe66.oe66 (.text:ti_sysbios_heaps_HeapMem_Module_GateProxy_leave__E)
                  8000c140    00000020     sysbios.ae66 : BIOS.obj (.text:ti_sysbios_heaps_HeapMem_isBlocking__E)
                  8000c160    00000020     app_pe66.oe66 (.text:ti_sysbios_knl_Clock_TimerProxy_Module__startupDone__S)
                  8000c180    00000020     app_pe66.oe66 (.text:ti_sysbios_knl_Clock_TimerProxy_getMaxTicks__E)
                  8000c1a0    00000020     sysbios.ae66 : BIOS.obj (.text:ti_sysbios_knl_Idle_loop__E)
                  8000c1c0    00000020                  : BIOS.obj (.text:ti_sysbios_knl_Queue_Instance_init__E)
                  8000c1e0    00000020     app_pe66.oe66 (.text:ti_sysbios_knl_Queue_Object__get__S)
                  8000c200    00000020     app_pe66.oe66 (.text:ti_sysbios_knl_Queue_destruct)
                  8000c220    00000020     sysbios.ae66 : BIOS.obj (.text:ti_sysbios_knl_Queue_empty__E)
                  8000c240    00000020                  : BIOS.obj (.text:ti_sysbios_knl_Semaphore_Instance_finalize__E)
                  8000c260    00000020     app_pe66.oe66 (.text:ti_sysbios_knl_Semaphore_destruct)
                  8000c280    00000020     sysbios.ae66 : BIOS.obj (.text:ti_sysbios_knl_Swi_disable__E)
                  8000c2a0    00000020     app_pe66.oe66 (.text:ti_sysbios_knl_Task_SupportProxy_Module__startupDone__S)
                  8000c2c0    00000020     sysbios.ae66 : BIOS.obj (.text:ti_sysbios_knl_Task_disable__E)
                  8000c2e0    00000020                  : BIOS.obj (.text:ti_sysbios_knl_Task_startup__E)
                  8000c300    00000020     app_pe66.oe66 (.text:ti_sysbios_timers_dmtimer_Timer_TimerSupportProxy_Module__startupDone__S)
                  8000c320    00000020     sysbios.ae66 : BIOS.obj (.text:ti_sysbios_timers_dmtimer_Timer_getMaxTicks__E)
                  8000c340    00000020     ti.targets.rts6000.ae66 : Error.oe66 (.text:xdc_runtime_Error_getSite__E)
                  8000c360    00000020                             : Error.oe66 (.text:xdc_runtime_Error_raiseX__E)
                  8000c380    00000020                             : Gate.oe66 (.text:xdc_runtime_Gate_enterSystem__E)
                  8000c3a0    00000020                             : Gate.oe66 (.text:xdc_runtime_Gate_leaveSystem__E)
                  8000c3c0    00000020     app_pe66.oe66 (.text:xdc_runtime_IHeap_alloc)
                  8000c3e0    00000020     app_pe66.oe66 (.text:xdc_runtime_IHeap_free)
                  8000c400    00000020     app_pe66.oe66 (.text:xdc_runtime_LoggerBuf_Module_GateProxy_enter__E)
                  8000c420    00000020     app_pe66.oe66 (.text:xdc_runtime_LoggerBuf_Module_GateProxy_leave__E)
                  8000c440    00000020     ti.targets.rts6000.ae66 : LoggerBuf.oe66 (.text:xdc_runtime_LoggerBuf_disable__E)
                  8000c460    00000020                             : LoggerBuf.oe66 (.text:xdc_runtime_LoggerBuf_enable__E)
                  8000c480    00000020                             : LoggerBuf.oe66 (.text:xdc_runtime_LoggerBuf_write1__E)
                  8000c4a0    00000020                             : LoggerBuf.oe66 (.text:xdc_runtime_LoggerBuf_write2__E)
                  8000c4c0    00000020     app_pe66.oe66 (.text:xdc_runtime_Memory_HeapProxy_alloc__E)
                  8000c4e0    00000020     app_pe66.oe66 (.text:xdc_runtime_Memory_HeapProxy_free__E)
                  8000c500    00000020     ti.targets.rts6000.ae66 : Memory.oe66 (.text:xdc_runtime_Memory_calloc__E)
                  8000c520    00000020                             : Memory.oe66 (.text:xdc_runtime_Memory_getMaxDefaultTypeAlign__E)
                  8000c540    00000020     app_pe66.oe66 (.text:xdc_runtime_Startup_exec__I)
                  8000c560    00000020     ti.targets.rts6000.ae66 : Startup.oe66 (.text:xdc_runtime_Startup_rtsDone__E)
                  8000c580    00000020                             : SysMin.oe66 (.text:xdc_runtime_SysMin_ready__E)
                  8000c5a0    00000020     app_pe66.oe66 (.text:xdc_runtime_System_Module_GateProxy_enter__E)
                  8000c5c0    00000020     app_pe66.oe66 (.text:xdc_runtime_System_Module_GateProxy_leave__E)
                  8000c5e0    00000020     ti.targets.rts6000.ae66 : System.oe66 (.text:xdc_runtime_System_Module_startup__E)
                  8000c600    00000020                             : System.oe66 (.text:xdc_runtime_System_aprintf_va__F)
                  8000c620    00000020                             : System.oe66 (.text:xdc_runtime_System_printf_va__F)
                  8000c640    00000020                             : System.oe66 (.text:xdc_runtime_System_vsnprintf__E)
                  8000c660    00000020     app_pe66.oe66 (.text:xdc_runtime_Text_visitRope__I)

.const     0    8000c680    00002d8a     
                  8000c680    00001ca4     app_pe66.oe66 (.const:xdc_runtime_Text_charTab__A)
                  8000e324    00000518     sysbios.ae66 : BIOS.obj (.const:.string)
                  8000e83c    00000004     ti.targets.rts6000.ae66 : Assert.oe66 (.const:.string)
                  8000e840    00000400     app_pe66.oe66 (.const:ti_sysbios_family_c66_Cache_marvalues__C)
                  8000ec40    000000dc     app_pe66.oe66 (.const:xdc_runtime_Text_nodeTab__A)
                  8000ed1c    00000064     app_pe66.oe66 (.const:.string)
                  8000ed80    00000058     ti.targets.rts6000.ae66 : Error.oe66 (.const:.string)
                  8000edd8    0000004c     main.obj (.const:.string)
                  8000ee24    00000040     ti.targets.rts6000.ae66 : Text.oe66 (.const:.string)
                  8000ee64    0000003c     app_pe66.oe66 (.const:ti_sysbios_knl_Task_Object__PARAMS__C)
                  8000eea0    0000003c     app_pe66.oe66 (.const:xdc_runtime_LoggerBuf_Module__FXNS__C)
                  8000eedc    00000004     app_pe66.oe66 (.const:ti_sysbios_family_c62_TaskSupport_stackAlignment__C)
                  8000eee0    00000034     app_pe66.oe66 (.const:xdc_runtime_Startup_sfxnTab__A)
                  8000ef14    0000002c     ti.targets.rts6000.ae66 : Startup.oe66 (.const:.string)
                  8000ef40    00000028     app_pe66.oe66 (.const:ti_sysbios_heaps_HeapMem_Module__FXNS__C)
                  8000ef68    00000028     app_pe66.oe66 (.const:xdc_runtime_LoggerBuf_Object__PARAMS__C)
                  8000ef90    00000024     app_pe66.oe66 (.const:ti_sysbios_gates_GateHwi_Module__FXNS__C)
                  8000efb4    00000024     app_pe66.oe66 (.const:ti_sysbios_gates_GateMutex_Module__FXNS__C)
                  8000efd8    00000024     app_pe66.oe66 (.const:ti_sysbios_heaps_HeapMem_Object__PARAMS__C)
                  8000effc    00000024     app_pe66.oe66 (.const:ti_sysbios_knl_Semaphore_Object__PARAMS__C)
                  8000f020    00000020     app_pe66.oe66 (.const:ti_sysbios_gates_GateHwi_Object__DESC__C)
                  8000f040    00000020     app_pe66.oe66 (.const:ti_sysbios_gates_GateMutex_Object__DESC__C)
                  8000f060    00000020     app_pe66.oe66 (.const:ti_sysbios_heaps_HeapMem_Object__DESC__C)
                  8000f080    00000020     app_pe66.oe66 (.const:ti_sysbios_knl_Queue_Object__DESC__C)
                  8000f0a0    00000020     app_pe66.oe66 (.const:ti_sysbios_knl_Semaphore_Object__DESC__C)
                  8000f0c0    00000020     app_pe66.oe66 (.const:ti_sysbios_knl_Task_Object__DESC__C)
                  8000f0e0    00000020     app_pe66.oe66 (.const:xdc_runtime_LoggerBuf_Object__DESC__C)
                  8000f100    0000001a     app_pe66.oe66 (.const:xdc_runtime_Startup_sfxnRts__A)
                  8000f11a    00000002     app_pe66.oe66 (.const:ti_sysbios_family_c64p_Exception_Module__id__C)
                  8000f11c    00000018     app_pe66.oe66 (.const:ti_sysbios_gates_GateHwi_Object__PARAMS__C)
                  8000f134    00000018     app_pe66.oe66 (.const:ti_sysbios_gates_GateMutex_Object__PARAMS__C)
                  8000f14c    00000018     app_pe66.oe66 (.const:ti_sysbios_knl_Queue_Object__PARAMS__C)
                  8000f164    00000004     app_pe66.oe66 (.const:ti_sysbios_family_c64p_Exception_E_exceptionMax__C)
                  8000f168    00000011     ti.targets.rts6000.ae66 : System.oe66 (.const:.string:digtohex)
                  8000f179    00000001     --HOLE-- [fill = 0]
                  8000f17a    00000002     app_pe66.oe66 (.const:ti_sysbios_family_c64p_Exception_useInternalBuffer__C)
                  8000f17c    00000008     ti.targets.rts6000.ae66 : System.oe66 (.const:.string)
                  8000f184    00000008     app_pe66.oe66 (.const:ti_sysbios_knl_Idle_funcList__C)
                  8000f18c    00000004     app_pe66.oe66 (.const:ti_sysbios_family_c64p_Exception_exceptionHook__C)
                  8000f190    00000008     app_pe66.oe66 (.const:xdc_runtime_Startup_firstFxns__A)
                  8000f198    00000008     app_pe66.oe66 (.const:xdc_runtime_Startup_firstFxns__C)
                  8000f1a0    00000008     app_pe66.oe66 (.const:xdc_runtime_Startup_lastFxns__C)
                  8000f1a8    00000004     app_pe66.oe66 (.const:ti_sysbios_family_c64p_Exception_externalHook__C)
                  8000f1ac    00000004     app_pe66.oe66 (.const:ti_sysbios_family_c64p_Exception_internalHook__C)
                  8000f1b0    00000004     app_pe66.oe66 (.const:ti_sysbios_family_c64p_Exception_nmiHook__C)
                  8000f1b4    00000004     app_pe66.oe66 (.const:ti_sysbios_family_c64p_Hwi_LD_end__C)
                  8000f1b8    00000004     app_pe66.oe66 (.const:ti_sysbios_family_c64p_Hwi_LM_begin__C)
                  8000f1bc    00000004     app_pe66.oe66 (.const:ti_sysbios_family_c64p_Hwi_Module__diagsEnabled__C)
                  8000f1c0    00000004     app_pe66.oe66 (.const:ti_sysbios_family_c64p_Hwi_Module__diagsIncluded__C)
                  8000f1c4    00000004     app_pe66.oe66 (.const:ti_sysbios_family_c64p_Hwi_Module__diagsMask__C)
                  8000f1c8    00000004     app_pe66.oe66 (.const:ti_sysbios_family_c64p_Hwi_Module__loggerFxn1__C)
                  8000f1cc    00000004     app_pe66.oe66 (.const:ti_sysbios_family_c64p_Hwi_Module__loggerFxn8__C)
                  8000f1d0    00000004     app_pe66.oe66 (.const:ti_sysbios_family_c64p_Hwi_Module__loggerObj__C)
                  8000f1d4    00000004     app_pe66.oe66 (.const:ti_sysbios_family_c66_Cache_E_invalidL1CacheSize__C)
                  8000f1d8    00000004     app_pe66.oe66 (.const:ti_sysbios_family_c66_Cache_E_invalidL2CacheSize__C)
                  8000f1dc    00000004     app_pe66.oe66 (.const:ti_sysbios_family_c66_Cache_atomicBlockSize__C)
                  8000f1e0    00000004     app_pe66.oe66 (.const:ti_sysbios_gates_GateMutex_A_badContext__C)
                  8000f1e4    00000004     app_pe66.oe66 (.const:ti_sysbios_gates_GateMutex_Instance_State_sem__O)
                  8000f1e8    00000004     app_pe66.oe66 (.const:ti_sysbios_gates_GateMutex_Module__diagsEnabled__C)
                  8000f1ec    00000004     app_pe66.oe66 (.const:ti_sysbios_gates_GateMutex_Module__diagsIncluded__C)
                  8000f1f0    00000004     app_pe66.oe66 (.const:ti_sysbios_gates_GateMutex_Module__diagsMask__C)
                  8000f1f4    00000004     app_pe66.oe66 (.const:ti_sysbios_hal_Hwi_E_stackOverflow__C)
                  8000f1f8    00000004     app_pe66.oe66 (.const:ti_sysbios_heaps_HeapMem_A_align__C)
                  8000f1fc    00000004     app_pe66.oe66 (.const:ti_sysbios_heaps_HeapMem_A_heapSize__C)
                  8000f200    00000004     app_pe66.oe66 (.const:ti_sysbios_heaps_HeapMem_A_invalidFree__C)
                  8000f204    00000004     app_pe66.oe66 (.const:ti_sysbios_heaps_HeapMem_A_zeroBlock__C)
                  8000f208    00000004     app_pe66.oe66 (.const:ti_sysbios_heaps_HeapMem_E_memory__C)
                  8000f20c    00000004     app_pe66.oe66 (.const:ti_sysbios_heaps_HeapMem_Module__diagsEnabled__C)
                  8000f210    00000004     app_pe66.oe66 (.const:ti_sysbios_heaps_HeapMem_Module__diagsIncluded__C)
                  8000f214    00000004     app_pe66.oe66 (.const:ti_sysbios_heaps_HeapMem_Module__diagsMask__C)
                  8000f218    00000004     app_pe66.oe66 (.const:ti_sysbios_heaps_HeapMem_Module__gateObj__C)
                  8000f21c    00000004     app_pe66.oe66 (.const:ti_sysbios_heaps_HeapMem_Object__count__C)
                  8000f220    00000004     app_pe66.oe66 (.const:ti_sysbios_heaps_HeapMem_reqAlign__C)
                  8000f224    00000004     app_pe66.oe66 (.const:ti_sysbios_knl_Clock_LM_begin__C)
                  8000f228    00000004     app_pe66.oe66 (.const:ti_sysbios_knl_Clock_LM_tick__C)
                  8000f22c    00000004     app_pe66.oe66 (.const:ti_sysbios_knl_Clock_LW_delayed__C)
                  8000f230    00000004     app_pe66.oe66 (.const:ti_sysbios_knl_Clock_Module_State_clockQ__O)
                  8000f234    00000004     app_pe66.oe66 (.const:ti_sysbios_knl_Clock_Module__diagsEnabled__C)
                  8000f238    00000004     app_pe66.oe66 (.const:ti_sysbios_knl_Clock_Module__diagsIncluded__C)
                  8000f23c    00000004     app_pe66.oe66 (.const:ti_sysbios_knl_Clock_Module__diagsMask__C)
                  8000f240    00000004     app_pe66.oe66 (.const:ti_sysbios_knl_Clock_Module__loggerFxn1__C)
                  8000f244    00000004     app_pe66.oe66 (.const:ti_sysbios_knl_Clock_Module__loggerFxn2__C)
                  8000f248    00000004     app_pe66.oe66 (.const:ti_sysbios_knl_Clock_Module__loggerObj__C)
                  8000f24c    00000004     app_pe66.oe66 (.const:ti_sysbios_knl_Semaphore_A_badContext__C)
                  8000f250    00000004     app_pe66.oe66 (.const:ti_sysbios_knl_Idle_funcList__A)
                  8000f254    00000004     app_pe66.oe66 (.const:ti_sysbios_knl_Semaphore_A_noEvents__C)
                  8000f258    00000004     app_pe66.oe66 (.const:ti_sysbios_knl_Semaphore_A_overflow__C)
                  8000f25c    00000004     app_pe66.oe66 (.const:ti_sysbios_knl_Semaphore_A_pendTaskDisabled__C)
                  8000f260    00000004     app_pe66.oe66 (.const:ti_sysbios_knl_Semaphore_Instance_State_pendQ__O)
                  8000f264    00000004     app_pe66.oe66 (.const:ti_sysbios_knl_Semaphore_LM_pend__C)
                  8000f268    00000004     app_pe66.oe66 (.const:ti_sysbios_knl_Semaphore_LM_post__C)
                  8000f26c    00000004     app_pe66.oe66 (.const:ti_sysbios_knl_Semaphore_Module__diagsEnabled__C)
                  8000f270    00000004     app_pe66.oe66 (.const:ti_sysbios_knl_Semaphore_Module__diagsIncluded__C)
                  8000f274    00000004     app_pe66.oe66 (.const:ti_sysbios_knl_Semaphore_Module__diagsMask__C)
                  8000f278    00000004     app_pe66.oe66 (.const:ti_sysbios_knl_Semaphore_Module__loggerFxn2__C)
                  8000f27c    00000004     app_pe66.oe66 (.const:ti_sysbios_knl_Semaphore_Module__loggerFxn4__C)
                  8000f280    00000004     app_pe66.oe66 (.const:ti_sysbios_knl_Semaphore_Module__loggerObj__C)
                  8000f284    00000004     app_pe66.oe66 (.const:ti_sysbios_knl_Swi_LD_end__C)
                  8000f288    00000004     app_pe66.oe66 (.const:ti_sysbios_knl_Swi_LM_begin__C)
                  8000f28c    00000004     app_pe66.oe66 (.const:ti_sysbios_knl_Swi_LM_post__C)
                  8000f290    00000004     app_pe66.oe66 (.const:ti_sysbios_knl_Swi_Module__diagsEnabled__C)
                  8000f294    00000004     app_pe66.oe66 (.const:ti_sysbios_knl_Swi_Module__diagsIncluded__C)
                  8000f298    00000004     app_pe66.oe66 (.const:ti_sysbios_knl_Swi_Module__diagsMask__C)
                  8000f29c    00000004     app_pe66.oe66 (.const:ti_sysbios_knl_Swi_Module__loggerFxn1__C)
                  8000f2a0    00000004     app_pe66.oe66 (.const:ti_sysbios_knl_Swi_Module__loggerFxn4__C)
                  8000f2a4    00000004     app_pe66.oe66 (.const:ti_sysbios_knl_Swi_Module__loggerObj__C)
                  8000f2a8    00000004     app_pe66.oe66 (.const:ti_sysbios_knl_Swi_Object__count__C)
                  8000f2ac    00000004     app_pe66.oe66 (.const:ti_sysbios_knl_Task_A_badPriority__C)
                  8000f2b0    00000004     app_pe66.oe66 (.const:ti_sysbios_knl_Task_A_badTaskState__C)
                  8000f2b4    00000004     app_pe66.oe66 (.const:ti_sysbios_knl_Task_A_badThreadType__C)
                  8000f2b8    00000004     app_pe66.oe66 (.const:ti_sysbios_knl_Task_A_badTimeout__C)
                  8000f2bc    00000004     app_pe66.oe66 (.const:ti_sysbios_knl_Task_A_noPendElem__C)
                  8000f2c0    00000004     app_pe66.oe66 (.const:ti_sysbios_knl_Task_A_sleepTaskDisabled__C)
                  8000f2c4    00000004     app_pe66.oe66 (.const:ti_sysbios_knl_Task_E_spOutOfBounds__C)
                  8000f2c8    00000004     app_pe66.oe66 (.const:ti_sysbios_knl_Task_E_stackOverflow__C)
                  8000f2cc    00000004     app_pe66.oe66 (.const:ti_sysbios_knl_Task_LD_block__C)
                  8000f2d0    00000004     app_pe66.oe66 (.const:ti_sysbios_knl_Task_LD_exit__C)
                  8000f2d4    00000004     app_pe66.oe66 (.const:ti_sysbios_knl_Task_LD_ready__C)
                  8000f2d8    00000004     app_pe66.oe66 (.const:ti_sysbios_knl_Task_LM_sleep__C)
                  8000f2dc    00000004     app_pe66.oe66 (.const:ti_sysbios_knl_Task_LM_switch__C)
                  8000f2e0    00000004     app_pe66.oe66 (.const:ti_sysbios_knl_Task_Module_State_inactiveQ__O)
                  8000f2e4    00000004     app_pe66.oe66 (.const:ti_sysbios_knl_Task_Module__diagsEnabled__C)
                  8000f2e8    00000004     app_pe66.oe66 (.const:ti_sysbios_knl_Task_Module__diagsIncluded__C)
                  8000f2ec    00000004     app_pe66.oe66 (.const:ti_sysbios_knl_Task_Module__diagsMask__C)
                  8000f2f0    00000004     app_pe66.oe66 (.const:ti_sysbios_knl_Task_Module__loggerFxn2__C)
                  8000f2f4    00000004     app_pe66.oe66 (.const:ti_sysbios_knl_Task_Module__loggerFxn4__C)
                  8000f2f8    00000004     app_pe66.oe66 (.const:ti_sysbios_knl_Task_Module__loggerObj__C)
                  8000f2fc    00000004     app_pe66.oe66 (.const:ti_sysbios_knl_Task_Object__count__C)
                  8000f300    00000004     app_pe66.oe66 (.const:ti_sysbios_knl_Task_allBlockedFunc__C)
                  8000f304    00000004     app_pe66.oe66 (.const:ti_sysbios_knl_Task_defaultStackHeap__C)
                  8000f308    00000004     app_pe66.oe66 (.const:ti_sysbios_knl_Task_defaultStackSize__C)
                  8000f30c    00000004     app_pe66.oe66 (.const:ti_sysbios_knl_Task_numConstructedTasks__C)
                  8000f310    00000004     app_pe66.oe66 (.const:ti_sysbios_timers_dmtimer_Timer_E_cannotSupport__C)
                  8000f314    00000004     app_pe66.oe66 (.const:ti_sysbios_timers_dmtimer_Timer_E_freqMismatch__C)
                  8000f318    00000004     app_pe66.oe66 (.const:ti_sysbios_timers_dmtimer_Timer_Module__diagsEnabled__C)
                  8000f31c    00000004     app_pe66.oe66 (.const:ti_sysbios_timers_dmtimer_Timer_Module__diagsIncluded__C)
                  8000f320    00000004     app_pe66.oe66 (.const:ti_sysbios_timers_dmtimer_Timer_Module__diagsMask__C)
                  8000f324    00000004     app_pe66.oe66 (.const:ti_sysbios_timers_dmtimer_Timer_numTimerDevices__C)
                  8000f328    00000004     app_pe66.oe66 (.const:xdc_runtime_Assert_E_assertFailed__C)
                  8000f32c    00000004     app_pe66.oe66 (.const:xdc_runtime_Core_A_initializedParams__C)
                  8000f330    00000004     app_pe66.oe66 (.const:xdc_runtime_Core_Module__diagsEnabled__C)
                  8000f334    00000004     app_pe66.oe66 (.const:xdc_runtime_Core_Module__diagsIncluded__C)
                  8000f338    00000004     app_pe66.oe66 (.const:xdc_runtime_Core_Module__diagsMask__C)
                  8000f33c    00000004     app_pe66.oe66 (.const:xdc_runtime_Error_E_memory__C)
                  8000f340    00000004     app_pe66.oe66 (.const:xdc_runtime_Error_Module__diagsEnabled__C)
                  8000f344    00000004     app_pe66.oe66 (.const:xdc_runtime_Error_Module__diagsIncluded__C)
                  8000f348    00000004     app_pe66.oe66 (.const:xdc_runtime_Error_Module__diagsMask__C)
                  8000f34c    00000004     app_pe66.oe66 (.const:xdc_runtime_Error_Module__loggerFxn8__C)
                  8000f350    00000004     app_pe66.oe66 (.const:xdc_runtime_Error_Module__loggerObj__C)
                  8000f354    00000004     app_pe66.oe66 (.const:xdc_runtime_Error_policyFxn__C)
                  8000f358    00000004     app_pe66.oe66 (.const:xdc_runtime_Error_policy__C)
                  8000f35c    00000004     app_pe66.oe66 (.const:xdc_runtime_Error_raiseHook__C)
                  8000f360    00000004     app_pe66.oe66 (.const:xdc_runtime_IFilterLogger_Interface__BASE__C)
                  8000f364    00000004     app_pe66.oe66 (.const:xdc_runtime_IGateProvider_Interface__BASE__C)
                  8000f368    00000004     app_pe66.oe66 (.const:xdc_runtime_IHeap_Interface__BASE__C)
                  8000f36c    00000004     app_pe66.oe66 (.const:xdc_runtime_ILogger_Interface__BASE__C)
                  8000f370    00000004     app_pe66.oe66 (.const:xdc_runtime_IModule_Interface__BASE__C)
                  8000f374    00000004     app_pe66.oe66 (.const:xdc_runtime_Log_L_error__C)
                  8000f378    00000004     app_pe66.oe66 (.const:xdc_runtime_LoggerBuf_E_badLevel__C)
                  8000f37c    00000004     app_pe66.oe66 (.const:xdc_runtime_LoggerBuf_Module__gateObj__C)
                  8000f380    00000004     app_pe66.oe66 (.const:xdc_runtime_LoggerBuf_Object__count__C)
                  8000f384    00000004     app_pe66.oe66 (.const:xdc_runtime_LoggerBuf_statusLogger__C)
                  8000f388    00000004     app_pe66.oe66 (.const:xdc_runtime_Memory_defaultHeapInstance__C)
                  8000f38c    00000004     app_pe66.oe66 (.const:xdc_runtime_Startup_execImpl__C)
                  8000f390    00000004     app_pe66.oe66 (.const:xdc_runtime_Startup_maxPasses__C)
                  8000f394    00000004     app_pe66.oe66 (.const:xdc_runtime_Startup_sfxnRts__C)
                  8000f398    00000004     app_pe66.oe66 (.const:xdc_runtime_Startup_sfxnTab__C)
                  8000f39c    00000004     app_pe66.oe66 (.const:xdc_runtime_SysMin_bufSize__C)
                  8000f3a0    00000004     app_pe66.oe66 (.const:xdc_runtime_SysMin_outputFunc__C)
                  8000f3a4    00000004     app_pe66.oe66 (.const:xdc_runtime_System_Module__gateObj__C)
                  8000f3a8    00000004     app_pe66.oe66 (.const:xdc_runtime_System_abortFxn__C)
                  8000f3ac    00000004     app_pe66.oe66 (.const:xdc_runtime_System_exitFxn__C)
                  8000f3b0    00000004     app_pe66.oe66 (.const:xdc_runtime_System_extendFxn__C)
                  8000f3b4    00000004     app_pe66.oe66 (.const:xdc_runtime_System_maxAtexitHandlers__C)
                  8000f3b8    00000004     app_pe66.oe66 (.const:xdc_runtime_Text_charTab__C)
                  8000f3bc    00000004     app_pe66.oe66 (.const:xdc_runtime_Text_nameEmpty__C)
                  8000f3c0    00000004     app_pe66.oe66 (.const:xdc_runtime_Text_nameStatic__C)
                  8000f3c4    00000004     app_pe66.oe66 (.const:xdc_runtime_Text_nameUnknown__C)
                  8000f3c8    00000004     app_pe66.oe66 (.const:xdc_runtime_Text_nodeTab__C)
                  8000f3cc    00000004     app_pe66.oe66 (.const:xdc_runtime_Text_visitRopeFxn__C)
                  8000f3d0    00000002     app_pe66.oe66 (.const:ti_sysbios_family_c64p_Hwi_Module__id__C)
                  8000f3d2    00000002     app_pe66.oe66 (.const:ti_sysbios_family_c64p_Hwi_Module__loggerDefined__C)
                  8000f3d4    00000002     app_pe66.oe66 (.const:ti_sysbios_family_c66_Cache_Module__id__C)
                  8000f3d6    00000002     app_pe66.oe66 (.const:ti_sysbios_family_c66_Cache_registerRTSSynch__C)
                  8000f3d8    00000002     app_pe66.oe66 (.const:ti_sysbios_gates_GateMutex_Module__id__C)
                  8000f3da    00000002     app_pe66.oe66 (.const:ti_sysbios_hal_Hwi_Module__id__C)
                  8000f3dc    00000002     app_pe66.oe66 (.const:ti_sysbios_heaps_HeapMem_Module__id__C)
                  8000f3de    00000002     app_pe66.oe66 (.const:ti_sysbios_knl_Clock_Module__id__C)
                  8000f3e0    00000002     app_pe66.oe66 (.const:ti_sysbios_knl_Clock_Module__loggerDefined__C)
                  8000f3e2    00000002     app_pe66.oe66 (.const:ti_sysbios_knl_Semaphore_Module__id__C)
                  8000f3e4    00000002     app_pe66.oe66 (.const:ti_sysbios_knl_Semaphore_Module__loggerDefined__C)
                  8000f3e6    00000002     app_pe66.oe66 (.const:ti_sysbios_knl_Swi_Module__id__C)
                  8000f3e8    00000002     app_pe66.oe66 (.const:ti_sysbios_knl_Swi_Module__loggerDefined__C)
                  8000f3ea    00000002     app_pe66.oe66 (.const:ti_sysbios_knl_Task_Module__id__C)
                  8000f3ec    00000002     app_pe66.oe66 (.const:ti_sysbios_knl_Task_Module__loggerDefined__C)
                  8000f3ee    00000002     app_pe66.oe66 (.const:ti_sysbios_timers_dmtimer_Timer_Module__id__C)
                  8000f3f0    00000002     app_pe66.oe66 (.const:ti_sysbios_timers_dmtimer_Timer_checkFrequency__C)
                  8000f3f2    00000002     app_pe66.oe66 (.const:ti_sysbios_timers_dmtimer_Timer_startupNeeded__C)
                  8000f3f4    00000002     app_pe66.oe66 (.const:xdc_runtime_Core_Module__id__C)
                  8000f3f6    00000002     app_pe66.oe66 (.const:xdc_runtime_Error_Module__loggerDefined__C)
                  8000f3f8    00000002     app_pe66.oe66 (.const:xdc_runtime_Error_maxDepth__C)
                  8000f3fa    00000002     app_pe66.oe66 (.const:xdc_runtime_LoggerBuf_Module__id__C)
                  8000f3fc    00000002     app_pe66.oe66 (.const:xdc_runtime_LoggerBuf_filterByLevel__C)
                  8000f3fe    00000002     app_pe66.oe66 (.const:xdc_runtime_Memory_Module__id__C)
                  8000f400    00000002     app_pe66.oe66 (.const:xdc_runtime_SysMin_flushAtExit__C)
                  8000f402    00000002     app_pe66.oe66 (.const:xdc_runtime_Text_charCnt__C)
                  8000f404    00000002     app_pe66.oe66 (.const:xdc_runtime_Text_isLoaded__C)
                  8000f406    00000002     app_pe66.oe66 (.const:xdc_runtime_Text_registryModsLastId__C)
                  8000f408    00000002     app_pe66.oe66 (.const:xdc_runtime_Text_unnamedModsLastId__C)

.stack     0    8000f410    00002000     UNINITIALIZED
                  8000f410    00000008     boot.ae66 : boot.oe66 (.stack)
                  8000f418    00001ff8     --HOLE--

.far       0    80011410    00001c08     UNINITIALIZED
                  80011410    00001400     app_pe66.oe66 (.far)
                  80012810    00000800     app_pe66.oe66 (.far:taskStackSection)
                  80013010    00000008     rts6600_elf.lib : trgdrv.obj (.far)

.fardata   0    80013018    00000644     
                  80013018    0000020c     app_pe66.oe66 (.fardata)
                  80013224    00000004     --HOLE--
                  80013228    000000c0     app_pe66.oe66 (.fardata:ti_sysbios_timers_dmtimer_Timer_Module_State_0_device__A)
                  800132e8    00000080     app_pe66.oe66 (.fardata:ti_sysbios_knl_Swi_Module_State_0_readyQ__A)
                  80013368    00000080     app_pe66.oe66 (.fardata:ti_sysbios_knl_Task_Module_State_0_readyQ__A)
                  800133e8    00000080     app_pe66.oe66 (.fardata:ti_sysbios_timers_dmtimer_Timer_Module_State_0_intFreqs__A)
                  80013468    00000060     app_pe66.oe66 (.fardata:ti_sysbios_timers_dmtimer_Timer_Object__table__V)
                  800134c8    0000004c     app_pe66.oe66 (.fardata:ti_sysbios_knl_Task_Object__table__V)
                  80013514    00000004     --HOLE--
                  80013518    00000040     app_pe66.oe66 (.fardata:ti_sysbios_gates_GateMutex_Object__table__V)
                  80013558    00000040     app_pe66.oe66 (.fardata:ti_sysbios_timers_dmtimer_Timer_Module_State_0_handles__A)
                  80013598    00000030     app_pe66.oe66 (.fardata:ti_sysbios_knl_Swi_Object__table__V)
                  800135c8    00000024     app_pe66.oe66 (.fardata:xdc_runtime_LoggerBuf_Object__table__V)
                  800135ec    00000004     --HOLE--
                  800135f0    00000018     app_pe66.oe66 (.fardata:ti_sysbios_family_c64p_Hwi_Object__table__V)
                  80013608    00000018     app_pe66.oe66 (.fardata:ti_sysbios_heaps_HeapMem_Object__table__V)
                  80013620    00000010     app_pe66.oe66 (.fardata:xdc_runtime_System_Module_State_0_atexitHandlers__A)
                  80013630    0000000c     rts6600_elf.lib : exit.obj (.fardata)
                  8001363c    00000008                     : _lock.obj (.fardata)
                  80013644    00000004     --HOLE--
                  80013648    00000008     app_pe66.oe66 (.fardata:ti_sysbios_hal_Hwi_Object__table__V)
                  80013650    00000004     app_pe66.oe66 (.fardata:ti_sysbios_gates_GateHwi_Object__table__V)
                  80013654    00000004     --HOLE--
                  80013658    00000004     app_pe66.oe66 (.fardata:ti_sysbios_knl_Task_Module_State_0_idleTask__A)

.cio       0    80013660    00000120     UNINITIALIZED
                  80013660    00000120     rts6600_elf.lib : trgmsg.obj (.cio)

.vecs      0    80013800    00000200     
                  80013800    00000200     app_pe66.oe66 (.vecs)

.cinit     0    80013a00    00000470     
                  80013a00    00000446     (.cinit..fardata.load) [load image, compression = rle]
                  80013e46    00000002     --HOLE-- [fill = 0]
                  80013e48    0000000c     (__TI_handler_table)
                  80013e54    00000008     (.cinit..far.load) [load image, compression = zero_init]
                  80013e5c    00000004     --HOLE-- [fill = 0]
                  80013e60    00000010     (__TI_cinit_table)


LINKER GENERATED COPY TABLES

__TI_cinit_table @ 80013e60 records: 2, size/record: 8, table size: 16
	.fardata: load addr=80013a00, load size=00000446 bytes, run addr=80013018, run size=00000644 bytes, compression=rle
	.far: load addr=80013e54, load size=00000008 bytes, run addr=80011410, run size=00001c08 bytes, compression=zero_init


LINKER GENERATED HANDLER TABLE

__TI_handler_table @ 80013e48 records: 3, size/record: 4, table size: 12
	index: 0, handler: __TI_decompress_rle24
	index: 1, handler: __TI_decompress_none
	index: 2, handler: __TI_zero_init


GLOBAL SYMBOLS: SORTED ALPHABETICALLY BY Name 

address    name
--------   ----
8000bcc0   C$$EXIT
8000af78   C$$IO$$
80008c20   HOSTwrite
8000bbe0   LoggerBuf_instanceStartup
80000000   __ASM__
80013660   __CIOBUF_
80000058   __ISA__
80000070   __PLAT__
80000098   __TARG__
80013e60   __TI_CINIT_Base
80013e70   __TI_CINIT_Limit
80013e48   __TI_Handler_Table_Base
80013e54   __TI_Handler_Table_Limit
UNDEFED    __TI_INITARRAY_Base
UNDEFED    __TI_INITARRAY_Limit
80011410   __TI_STACK_END
00002000   __TI_STACK_SIZE
00000000   __TI_STATIC_BASE
UNDEFED    __TI_TLS_INIT_Base
UNDEFED    __TI_TLS_INIT_Limit
00000001   __TI_args_main
8000bce0   __TI_decompress_none
8000bd00   __TI_decompress_rle24
80013638   __TI_enable_exit_profile_output
ffffffff   __TI_pprof_out_hndl
ffffffff   __TI_prof_data_size
ffffffff   __TI_prof_data_start
800093a0   __TI_tls_init
80008520   __TI_zero_init
800000c0   __TRDR__
ffffffff   __binit__
80008ce0   __c6xabi_divu
800048c0   __c6xabi_divull
80009cc0   __c6xabi_llshl
8000a5c0   __c6xabi_llshru
800095e0   __c6xabi_remu
8000b220   __c6xabi_strasgi_64plus
ffffffff   __c_args__
80008ce0   __divu
800095e0   __remu
8000b220   __strasgi_64plus
8000bc00   __xdc__init
80013220   __xdc__init__addr
8000b260   _args_main
00000000   _argsize
80006fa0   _auto_init_elf
80009680   _c_int00
80013630   _cleanup_ptr
80013634   _dtors_ptr
8001363c   _lock
8000bc20   _nop
8000bc40   _register_lock
8000bc60   _register_synch_api
8000bc80   _register_unlock
8000f410   _stack
8000a620   _subcull
80013640   _unlock
8000bcc0   abort
ffffffff   binit
80008da0   exit
80008ea4   main
80009720   memcpy
80008600   memset
80009dc0   readmsg
80008e60   taskFxn
80013018   ti_sysbios_BIOS_Module__state__V
8000bd20   ti_sysbios_BIOS_RtsGateProxy_enter__E
8000bd40   ti_sysbios_BIOS_RtsGateProxy_leave__E
8000c0a0   ti_sysbios_BIOS_RtsGateProxy_query__E
8000a740   ti_sysbios_BIOS_atExitFunc__I
8000a7a0   ti_sysbios_BIOS_errorRaiseHook__I
8000b2e0   ti_sysbios_BIOS_exitFunc__I
8000bd60   ti_sysbios_BIOS_exit__E
8000bd80   ti_sysbios_BIOS_getCpuFreq__E
8000bda0   ti_sysbios_BIOS_linkedWithIncorrectBootLibrary__E
8000bdc0   ti_sysbios_BIOS_nullFunc__I
8000a800   ti_sysbios_BIOS_registerRTSLock__I
8000a860   ti_sysbios_BIOS_removeRTSLock__I
8000b320   ti_sysbios_BIOS_rtsLock__I
8000a8c0   ti_sysbios_BIOS_rtsUnlock__I
8000bde0   ti_sysbios_BIOS_setThreadType__E
8000a920   ti_sysbios_BIOS_startFunc__I
8000be00   ti_sysbios_BIOS_start__E
8000be20   ti_sysbios_family_c62_TaskSupport_Module__startupDone__S
8000b2a0   ti_sysbios_family_c62_TaskSupport_buildTaskStack
8000be40   ti_sysbios_family_c62_TaskSupport_checkStack__E
8000be60   ti_sysbios_family_c62_TaskSupport_getStackAlignment__E
8000bca0   ti_sysbios_family_c62_TaskSupport_glue
8000eedc   ti_sysbios_family_c62_TaskSupport_stackAlignment__C
8000a980   ti_sysbios_family_c62_TaskSupport_start__E
80009d40   ti_sysbios_family_c62_TaskSupport_swap__E
8000f164   ti_sysbios_family_c64p_Exception_E_exceptionMax__C
8000f11a   ti_sysbios_family_c64p_Exception_Module__id__C
8001303c   ti_sysbios_family_c64p_Exception_Module__state__V
800097c0   ti_sysbios_family_c64p_Exception_Module_startup__E
80006700   ti_sysbios_family_c64p_Exception_dispatch__E
8000f18c   ti_sysbios_family_c64p_Exception_exceptionHook__C
8000f1a8   ti_sysbios_family_c64p_Exception_externalHook__C
80000880   ti_sysbios_family_c64p_Exception_handler__I
80004b00   ti_sysbios_family_c64p_Exception_internalHandler__I
8000f1ac   ti_sysbios_family_c64p_Exception_internalHook__C
8000f1b0   ti_sysbios_family_c64p_Exception_nmiHook__C
8000f17a   ti_sysbios_family_c64p_Exception_useInternalBuffer__C
80013800   ti_sysbios_family_c64p_Hwi0
8000f1b4   ti_sysbios_family_c64p_Hwi_LD_end__C
8000f1b8   ti_sysbios_family_c64p_Hwi_LM_begin__C
8000f1bc   ti_sysbios_family_c64p_Hwi_Module__diagsEnabled__C
8000f1c0   ti_sysbios_family_c64p_Hwi_Module__diagsIncluded__C
8000f1c4   ti_sysbios_family_c64p_Hwi_Module__diagsMask__C
8000f3d0   ti_sysbios_family_c64p_Hwi_Module__id__C
8000f3d2   ti_sysbios_family_c64p_Hwi_Module__loggerDefined__C
8000f1c8   ti_sysbios_family_c64p_Hwi_Module__loggerFxn1__C
8000f1cc   ti_sysbios_family_c64p_Hwi_Module__loggerFxn8__C
8000f1d0   ti_sysbios_family_c64p_Hwi_Module__loggerObj__C
8001306c   ti_sysbios_family_c64p_Hwi_Module__root__V
8000b360   ti_sysbios_family_c64p_Hwi_Module__startupDone__F
8000b360   ti_sysbios_family_c64p_Hwi_Module__startupDone__S
80013074   ti_sysbios_family_c64p_Hwi_Module__state__V
800070e0   ti_sysbios_family_c64p_Hwi_Module_startup__E
800135f0   ti_sysbios_family_c64p_Hwi_Object__table__V
8000be80   ti_sysbios_family_c64p_Hwi_clearInterrupt__E
8000b3a0   ti_sysbios_family_c64p_Hwi_disableInterrupt__E
800053c0   ti_sysbios_family_c64p_Hwi_dispatchAlways
80009e40   ti_sysbios_family_c64p_Hwi_dispatchC__I
80004400   ti_sysbios_family_c64p_Hwi_dispatchCore__I
8000b3e0   ti_sysbios_family_c64p_Hwi_enableInterrupt__E
80009ec0   ti_sysbios_family_c64p_Hwi_getStackInfo__E
80013800   ti_sysbios_family_c64p_Hwi_int0
80013820   ti_sysbios_family_c64p_Hwi_int1
80013940   ti_sysbios_family_c64p_Hwi_int10
80013960   ti_sysbios_family_c64p_Hwi_int11
80013980   ti_sysbios_family_c64p_Hwi_int12
800139a0   ti_sysbios_family_c64p_Hwi_int13
800139c0   ti_sysbios_family_c64p_Hwi_int14
800139e0   ti_sysbios_family_c64p_Hwi_int15
80013840   ti_sysbios_family_c64p_Hwi_int2
80013860   ti_sysbios_family_c64p_Hwi_int3
80013880   ti_sysbios_family_c64p_Hwi_int4
800138a0   ti_sysbios_family_c64p_Hwi_int5
800138c0   ti_sysbios_family_c64p_Hwi_int6
800138e0   ti_sysbios_family_c64p_Hwi_int7
80013900   ti_sysbios_family_c64p_Hwi_int8
80013920   ti_sysbios_family_c64p_Hwi_int9
8000bea0   ti_sysbios_family_c64p_Hwi_startup__E
8000a680   ti_sysbios_family_c64p_Hwi_switchAndDispatch__I
8000bec0   ti_sysbios_family_c64p_Hwi_switchFromBootStack__E
8000bee0   ti_sysbios_family_c64p_TimestampProvider_Module_startup__E
8000bf00   ti_sysbios_family_c64p_TimestampProvider_get32__E
8000bf20   ti_sysbios_family_c64p_TimestampProvider_get64__E
8000bd80   ti_sysbios_family_c64p_TimestampProvider_getFreq__E
8000f1d4   ti_sysbios_family_c66_Cache_E_invalidL1CacheSize__C
8000f1d8   ti_sysbios_family_c66_Cache_E_invalidL2CacheSize__C
8000f3d4   ti_sysbios_family_c66_Cache_Module__id__C
8000a9e0   ti_sysbios_family_c66_Cache_Module_startup__E
8000bf40   ti_sysbios_family_c66_Cache_RTSSynchInv__I
8000bf60   ti_sysbios_family_c66_Cache_RTSSynchWbInv__I
8000bf80   ti_sysbios_family_c66_Cache_RTSSynchWb__I
8000f1dc   ti_sysbios_family_c66_Cache_atomicBlockSize__C
80005980   ti_sysbios_family_c66_Cache_block__I
80007720   ti_sysbios_family_c66_Cache_getL1DInitSize__I
80007840   ti_sysbios_family_c66_Cache_getL1PInitSize__I
80006b80   ti_sysbios_family_c66_Cache_getL2InitSize__I
00008000   ti_sysbios_family_c66_Cache_l1dSize
00008000   ti_sysbios_family_c66_Cache_l1pSize
00000000   ti_sysbios_family_c66_Cache_l2Size
8000e840   ti_sysbios_family_c66_Cache_marvalues__C
8000f3d6   ti_sysbios_family_c66_Cache_registerRTSSynch__C
80007220   ti_sysbios_family_c66_Cache_startup__I
8000bfa0   ti_sysbios_family_c66_Cache_wait__E
8000b420   ti_sysbios_family_shared_vayu_TimerSupport_Module__startupDone__F
8000b420   ti_sysbios_family_shared_vayu_TimerSupport_Module__startupDone__S
8000bfc0   ti_sysbios_family_shared_vayu_TimerSupport_Module_startup__E
8000bfe0   ti_sysbios_family_shared_vayu_TimerSupport_enable__E
8000a6e0   ti_sysbios_family_xxx_Hwi_switchAndRunFunc
8000b460   ti_sysbios_gates_GateHwi_Handle__label__S
8000c000   ti_sysbios_gates_GateHwi_Instance_init__E
8000ef90   ti_sysbios_gates_GateHwi_Module__FXNS__C
800130e0   ti_sysbios_gates_GateHwi_Module__root__V
8000f020   ti_sysbios_gates_GateHwi_Object__DESC__C
8000f11c   ti_sysbios_gates_GateHwi_Object__PARAMS__C
8000aa40   ti_sysbios_gates_GateHwi_Object__create__S
8000b4a0   ti_sysbios_gates_GateHwi_Object__delete__S
80013650   ti_sysbios_gates_GateHwi_Object__table__V
8000c020   ti_sysbios_gates_GateHwi_enter__E
8000c040   ti_sysbios_gates_GateHwi_leave__E
8000c060   ti_sysbios_gates_GateHwi_query__E
8000f1e0   ti_sysbios_gates_GateMutex_A_badContext__C
8000b4e0   ti_sysbios_gates_GateMutex_Handle__label__S
8000f1e4   ti_sysbios_gates_GateMutex_Instance_State_sem__O
8000c080   ti_sysbios_gates_GateMutex_Instance_finalize__E
8000b520   ti_sysbios_gates_GateMutex_Instance_init__E
8000efb4   ti_sysbios_gates_GateMutex_Module__FXNS__C
8000f1e8   ti_sysbios_gates_GateMutex_Module__diagsEnabled__C
8000f1ec   ti_sysbios_gates_GateMutex_Module__diagsIncluded__C
8000f1f0   ti_sysbios_gates_GateMutex_Module__diagsMask__C
8000f3d8   ti_sysbios_gates_GateMutex_Module__id__C
800130e8   ti_sysbios_gates_GateMutex_Module__root__V
8000f040   ti_sysbios_gates_GateMutex_Object__DESC__C
8000f134   ti_sysbios_gates_GateMutex_Object__PARAMS__C
8000aaa0   ti_sysbios_gates_GateMutex_Object__create__S
8000b560   ti_sysbios_gates_GateMutex_Object__delete__S
80013518   ti_sysbios_gates_GateMutex_Object__table__V
80006240   ti_sysbios_gates_GateMutex_enter__E
8000b5a0   ti_sysbios_gates_GateMutex_leave__E
8000c0a0   ti_sysbios_gates_GateMutex_query__E
8000f1f4   ti_sysbios_hal_Hwi_E_stackOverflow__C
8000c0c0   ti_sysbios_hal_Hwi_HwiProxy_Module__startupDone__S
8000be80   ti_sysbios_hal_Hwi_HwiProxy_clearInterrupt__E
8000b3a0   ti_sysbios_hal_Hwi_HwiProxy_disableInterrupt__E
8000b3e0   ti_sysbios_hal_Hwi_HwiProxy_enableInterrupt__E
80009ec0   ti_sysbios_hal_Hwi_HwiProxy_getStackInfo__E
8000bea0   ti_sysbios_hal_Hwi_HwiProxy_startup__E
8000bec0   ti_sysbios_hal_Hwi_HwiProxy_switchFromBootStack__E
8000f3da   ti_sysbios_hal_Hwi_Module__id__C
800130f0   ti_sysbios_hal_Hwi_Module__root__V
8000c0e0   ti_sysbios_hal_Hwi_Module_startup__E
80013648   ti_sysbios_hal_Hwi_Object__table__V
80009f40   ti_sysbios_hal_Hwi_checkStack
8000be80   ti_sysbios_hal_Hwi_clearInterrupt__E
8000b3a0   ti_sysbios_hal_Hwi_disableInterrupt__E
8000b3e0   ti_sysbios_hal_Hwi_enableInterrupt__E
80009ec0   ti_sysbios_hal_Hwi_getStackInfo__E
80009fc0   ti_sysbios_hal_Hwi_initStack
8000bea0   ti_sysbios_hal_Hwi_startup__E
8000f1f8   ti_sysbios_heaps_HeapMem_A_align__C
8000f1fc   ti_sysbios_heaps_HeapMem_A_heapSize__C
8000f200   ti_sysbios_heaps_HeapMem_A_invalidFree__C
8000f204   ti_sysbios_heaps_HeapMem_A_zeroBlock__C
8000f208   ti_sysbios_heaps_HeapMem_E_memory__C
8000b5e0   ti_sysbios_heaps_HeapMem_Handle__label__S
80011410   ti_sysbios_heaps_HeapMem_Instance_State_0_buf__A
800036a0   ti_sysbios_heaps_HeapMem_Instance_init__E
8000c100   ti_sysbios_heaps_HeapMem_Module_GateProxy_enter__E
8000c120   ti_sysbios_heaps_HeapMem_Module_GateProxy_leave__E
8000c0a0   ti_sysbios_heaps_HeapMem_Module_GateProxy_query__E
8000ef40   ti_sysbios_heaps_HeapMem_Module__FXNS__C
8000f20c   ti_sysbios_heaps_HeapMem_Module__diagsEnabled__C
8000f210   ti_sysbios_heaps_HeapMem_Module__diagsIncluded__C
8000f214   ti_sysbios_heaps_HeapMem_Module__diagsMask__C
8000f218   ti_sysbios_heaps_HeapMem_Module__gateObj__C
8000f3dc   ti_sysbios_heaps_HeapMem_Module__id__C
800130f8   ti_sysbios_heaps_HeapMem_Module__root__V
8000f060   ti_sysbios_heaps_HeapMem_Object__DESC__C
8000efd8   ti_sysbios_heaps_HeapMem_Object__PARAMS__C
8000f21c   ti_sysbios_heaps_HeapMem_Object__count__C
8000ab00   ti_sysbios_heaps_HeapMem_Object__create__S
8000b620   ti_sysbios_heaps_HeapMem_Object__delete__S
8000b660   ti_sysbios_heaps_HeapMem_Object__get__S
80013608   ti_sysbios_heaps_HeapMem_Object__table__V
80001780   ti_sysbios_heaps_HeapMem_allocUnprotected__E
80008f20   ti_sysbios_heaps_HeapMem_alloc__E
80001d60   ti_sysbios_heaps_HeapMem_freeUnprotected__E
8000ab60   ti_sysbios_heaps_HeapMem_free__E
80008fe0   ti_sysbios_heaps_HeapMem_getStats__E
80009860   ti_sysbios_heaps_HeapMem_init__I
8000c140   ti_sysbios_heaps_HeapMem_isBlocking__E
8000f220   ti_sysbios_heaps_HeapMem_reqAlign__C
8000f224   ti_sysbios_knl_Clock_LM_begin__C
8000f228   ti_sysbios_knl_Clock_LM_tick__C
8000f22c   ti_sysbios_knl_Clock_LW_delayed__C
8000f230   ti_sysbios_knl_Clock_Module_State_clockQ__O
8000f234   ti_sysbios_knl_Clock_Module__diagsEnabled__C
8000f238   ti_sysbios_knl_Clock_Module__diagsIncluded__C
8000f23c   ti_sysbios_knl_Clock_Module__diagsMask__C
8000f3de   ti_sysbios_knl_Clock_Module__id__C
8000f3e0   ti_sysbios_knl_Clock_Module__loggerDefined__C
8000f240   ti_sysbios_knl_Clock_Module__loggerFxn1__C
8000f244   ti_sysbios_knl_Clock_Module__loggerFxn2__C
8000f248   ti_sysbios_knl_Clock_Module__loggerObj__C
80013100   ti_sysbios_knl_Clock_Module__root__V
80013108   ti_sysbios_knl_Clock_Module__state__V
8000abc0   ti_sysbios_knl_Clock_Module_startup__E
8000c160   ti_sysbios_knl_Clock_TimerProxy_Module__startupDone__S
8000c180   ti_sysbios_knl_Clock_TimerProxy_getMaxTicks__E
800088a0   ti_sysbios_knl_Clock_TimerProxy_startup__E
8000ac20   ti_sysbios_knl_Clock_doTick__I
800090a0   ti_sysbios_knl_Clock_logTick__E
80003c60   ti_sysbios_knl_Clock_workFunc__E
8000f250   ti_sysbios_knl_Idle_funcList__A
8000f184   ti_sysbios_knl_Idle_funcList__C
8000c1a0   ti_sysbios_knl_Idle_loop__E
8000a040   ti_sysbios_knl_Idle_run__E
8000c1c0   ti_sysbios_knl_Queue_Instance_init__E
80013134   ti_sysbios_knl_Queue_Module__root__V
8000f080   ti_sysbios_knl_Queue_Object__DESC__C
8000f14c   ti_sysbios_knl_Queue_Object__PARAMS__C
8000b6a0   ti_sysbios_knl_Queue_Object__destruct__S
8000c1e0   ti_sysbios_knl_Queue_Object__get__S
8000ac80   ti_sysbios_knl_Queue_construct
8000c200   ti_sysbios_knl_Queue_destruct
8000c220   ti_sysbios_knl_Queue_empty__E
8000f24c   ti_sysbios_knl_Semaphore_A_badContext__C
8000f254   ti_sysbios_knl_Semaphore_A_noEvents__C
8000f258   ti_sysbios_knl_Semaphore_A_overflow__C
8000f25c   ti_sysbios_knl_Semaphore_A_pendTaskDisabled__C
8000f260   ti_sysbios_knl_Semaphore_Instance_State_pendQ__O
8000c240   ti_sysbios_knl_Semaphore_Instance_finalize__E
80007360   ti_sysbios_knl_Semaphore_Instance_init__E
8000f264   ti_sysbios_knl_Semaphore_LM_pend__C
8000f268   ti_sysbios_knl_Semaphore_LM_post__C
8000f26c   ti_sysbios_knl_Semaphore_Module__diagsEnabled__C
8000f270   ti_sysbios_knl_Semaphore_Module__diagsIncluded__C
8000f274   ti_sysbios_knl_Semaphore_Module__diagsMask__C
8000f3e2   ti_sysbios_knl_Semaphore_Module__id__C
8000f3e4   ti_sysbios_knl_Semaphore_Module__loggerDefined__C
8000f278   ti_sysbios_knl_Semaphore_Module__loggerFxn2__C
8000f27c   ti_sysbios_knl_Semaphore_Module__loggerFxn4__C
8000f280   ti_sysbios_knl_Semaphore_Module__loggerObj__C
8001313c   ti_sysbios_knl_Semaphore_Module__root__V
8000f0a0   ti_sysbios_knl_Semaphore_Object__DESC__C
8000effc   ti_sysbios_knl_Semaphore_Object__PARAMS__C
8000b6e0   ti_sysbios_knl_Semaphore_Object__destruct__S
8000ace0   ti_sysbios_knl_Semaphore_construct
8000c260   ti_sysbios_knl_Semaphore_destruct
8000ad40   ti_sysbios_knl_Semaphore_pendTimeout__I
80001000   ti_sysbios_knl_Semaphore_pend__E
80003f00   ti_sysbios_knl_Semaphore_post__E
8000f284   ti_sysbios_knl_Swi_LD_end__C
8000f288   ti_sysbios_knl_Swi_LM_begin__C
8000f28c   ti_sysbios_knl_Swi_LM_post__C
800132e8   ti_sysbios_knl_Swi_Module_State_0_readyQ__A
8000f290   ti_sysbios_knl_Swi_Module__diagsEnabled__C
8000f294   ti_sysbios_knl_Swi_Module__diagsIncluded__C
8000f298   ti_sysbios_knl_Swi_Module__diagsMask__C
8000f3e6   ti_sysbios_knl_Swi_Module__id__C
8000f3e8   ti_sysbios_knl_Swi_Module__loggerDefined__C
8000f29c   ti_sysbios_knl_Swi_Module__loggerFxn1__C
8000f2a0   ti_sysbios_knl_Swi_Module__loggerFxn4__C
8000f2a4   ti_sysbios_knl_Swi_Module__loggerObj__C
80013144   ti_sysbios_knl_Swi_Module__root__V
8001314c   ti_sysbios_knl_Swi_Module__state__V
8000ada0   ti_sysbios_knl_Swi_Module_startup__E
8000f2a8   ti_sysbios_knl_Swi_Object__count__C
8000b720   ti_sysbios_knl_Swi_Object__get__S
80013598   ti_sysbios_knl_Swi_Object__table__V
8000c280   ti_sysbios_knl_Swi_disable__E
80006ce0   ti_sysbios_knl_Swi_post__E
80008020   ti_sysbios_knl_Swi_restoreHwi__E
800086e0   ti_sysbios_knl_Swi_runLoop__I
80004f80   ti_sysbios_knl_Swi_run__I
80008120   ti_sysbios_knl_Swi_schedule__I
800087c0   ti_sysbios_knl_Swi_startup__E
8000f2ac   ti_sysbios_knl_Task_A_badPriority__C
8000f2b0   ti_sysbios_knl_Task_A_badTaskState__C
8000f2b4   ti_sysbios_knl_Task_A_badThreadType__C
8000f2b8   ti_sysbios_knl_Task_A_badTimeout__C
8000f2bc   ti_sysbios_knl_Task_A_noPendElem__C
8000f2c0   ti_sysbios_knl_Task_A_sleepTaskDisabled__C
8000f2c4   ti_sysbios_knl_Task_E_spOutOfBounds__C
8000f2c8   ti_sysbios_knl_Task_E_stackOverflow__C
80012810   ti_sysbios_knl_Task_Instance_State_0_stack__A
80002300   ti_sysbios_knl_Task_Instance_finalize__E
80002fc0   ti_sysbios_knl_Task_Instance_init__E
8000f2cc   ti_sysbios_knl_Task_LD_block__C
8000f2d0   ti_sysbios_knl_Task_LD_exit__C
8000f2d4   ti_sysbios_knl_Task_LD_ready__C
8000f2d8   ti_sysbios_knl_Task_LM_sleep__C
8000f2dc   ti_sysbios_knl_Task_LM_switch__C
80013658   ti_sysbios_knl_Task_Module_State_0_idleTask__A
80013368   ti_sysbios_knl_Task_Module_State_0_readyQ__A
8000f2e0   ti_sysbios_knl_Task_Module_State_inactiveQ__O
8000f2e4   ti_sysbios_knl_Task_Module__diagsEnabled__C
8000f2e8   ti_sysbios_knl_Task_Module__diagsIncluded__C
8000f2ec   ti_sysbios_knl_Task_Module__diagsMask__C
8000f3ea   ti_sysbios_knl_Task_Module__id__C
8000f3ec   ti_sysbios_knl_Task_Module__loggerDefined__C
8000f2f0   ti_sysbios_knl_Task_Module__loggerFxn2__C
8000f2f4   ti_sysbios_knl_Task_Module__loggerFxn4__C
8000f2f8   ti_sysbios_knl_Task_Module__loggerObj__C
80013168   ti_sysbios_knl_Task_Module__root__V
80013170   ti_sysbios_knl_Task_Module__state__V
80003980   ti_sysbios_knl_Task_Module_startup__E
8000f0c0   ti_sysbios_knl_Task_Object__DESC__C
8000ee64   ti_sysbios_knl_Task_Object__PARAMS__C
8000f2fc   ti_sysbios_knl_Task_Object__count__C
8000b760   ti_sysbios_knl_Task_Object__get__S
800134c8   ti_sysbios_knl_Task_Object__table__V
8000c2a0   ti_sysbios_knl_Task_SupportProxy_Module__startupDone__S
8000be40   ti_sysbios_knl_Task_SupportProxy_checkStack__E
8000be60   ti_sysbios_knl_Task_SupportProxy_getStackAlignment__E
8000a980   ti_sysbios_knl_Task_SupportProxy_start__E
80009d40   ti_sysbios_knl_Task_SupportProxy_swap__E
8000f300   ti_sysbios_knl_Task_allBlockedFunc__C
80009160   ti_sysbios_knl_Task_allBlockedFunction__I
800074a0   ti_sysbios_knl_Task_blockI__E
80005b40   ti_sysbios_knl_Task_checkStacks__E
80009220   ti_sysbios_knl_Task_create
8000f304   ti_sysbios_knl_Task_defaultStackHeap__C
8000f308   ti_sysbios_knl_Task_defaultStackSize__C
8000c2c0   ti_sysbios_knl_Task_disable__E
8000ae00   ti_sysbios_knl_Task_enter__I
80005d00   ti_sysbios_knl_Task_exit__E
8000f30c   ti_sysbios_knl_Task_numConstructedTasks__C
800075e0   ti_sysbios_knl_Task_postInit__I
8000ae60   ti_sysbios_knl_Task_processVitalTaskFlag__I
8000a0c0   ti_sysbios_knl_Task_restore__E
800063e0   ti_sysbios_knl_Task_schedule__I
8000b7a0   ti_sysbios_knl_Task_sleepTimeout__I
800027a0   ti_sysbios_knl_Task_sleep__E
80006880   ti_sysbios_knl_Task_startCore__E
8000c2e0   ti_sysbios_knl_Task_startup__E
80008220   ti_sysbios_knl_Task_unblockI__E
800131b4   ti_sysbios_rts_ti_ThreadLocalStorage_Module__state__V
8000f310   ti_sysbios_timers_dmtimer_Timer_E_cannotSupport__C
8000f314   ti_sysbios_timers_dmtimer_Timer_E_freqMismatch__C
80013228   ti_sysbios_timers_dmtimer_Timer_Module_State_0_device__A
80013558   ti_sysbios_timers_dmtimer_Timer_Module_State_0_handles__A
800133e8   ti_sysbios_timers_dmtimer_Timer_Module_State_0_intFreqs__A
8000f318   ti_sysbios_timers_dmtimer_Timer_Module__diagsEnabled__C
8000f31c   ti_sysbios_timers_dmtimer_Timer_Module__diagsIncluded__C
8000f320   ti_sysbios_timers_dmtimer_Timer_Module__diagsMask__C
8000f3ee   ti_sysbios_timers_dmtimer_Timer_Module__id__C
800131c0   ti_sysbios_timers_dmtimer_Timer_Module__root__V
8000b7e0   ti_sysbios_timers_dmtimer_Timer_Module__startupDone__F
8000b7e0   ti_sysbios_timers_dmtimer_Timer_Module__startupDone__S
800131c8   ti_sysbios_timers_dmtimer_Timer_Module__state__V
80007960   ti_sysbios_timers_dmtimer_Timer_Module_startup__E
80013468   ti_sysbios_timers_dmtimer_Timer_Object__table__V
8000c300   ti_sysbios_timers_dmtimer_Timer_TimerSupportProxy_Module__startupDone__S
8000bfe0   ti_sysbios_timers_dmtimer_Timer_TimerSupportProxy_enable__E
80002c20   ti_sysbios_timers_dmtimer_Timer_checkFreq__I
8000f3f0   ti_sysbios_timers_dmtimer_Timer_checkFrequency__C
80003340   ti_sysbios_timers_dmtimer_Timer_deviceConfig__I
8000c320   ti_sysbios_timers_dmtimer_Timer_getMaxTicks__E
80007a80   ti_sysbios_timers_dmtimer_Timer_initDevice__I
8000f324   ti_sysbios_timers_dmtimer_Timer_numTimerDevices__C
80004d40   ti_sysbios_timers_dmtimer_Timer_setPeriodMicroSecs__E
80006e40   ti_sysbios_timers_dmtimer_Timer_start__E
8000f3f2   ti_sysbios_timers_dmtimer_Timer_startupNeeded__C
800088a0   ti_sysbios_timers_dmtimer_Timer_startup__E
800092e0   ti_sysbios_timers_dmtimer_Timer_stop__E
8000aec0   ti_sysbios_timers_dmtimer_Timer_stub__E
8000af20   writemsg
8000f328   xdc_runtime_Assert_E_assertFailed__C
80009900   xdc_runtime_Assert_raise__I
8000f32c   xdc_runtime_Core_A_initializedParams__C
8000f330   xdc_runtime_Core_Module__diagsEnabled__C
8000f334   xdc_runtime_Core_Module__diagsIncluded__C
8000f338   xdc_runtime_Core_Module__diagsMask__C
8000f3f4   xdc_runtime_Core_Module__id__C
8000a140   xdc_runtime_Core_assignLabel__I
8000a1c0   xdc_runtime_Core_assignParams__I
80006a00   xdc_runtime_Core_constructObject__I
800051a0   xdc_runtime_Core_createObject__I
80007ba0   xdc_runtime_Core_deleteObject__I
8000f33c   xdc_runtime_Error_E_memory__C
8000f340   xdc_runtime_Error_Module__diagsEnabled__C
8000f344   xdc_runtime_Error_Module__diagsIncluded__C
8000f348   xdc_runtime_Error_Module__diagsMask__C
8000f3f6   xdc_runtime_Error_Module__loggerDefined__C
8000f34c   xdc_runtime_Error_Module__loggerFxn8__C
8000f350   xdc_runtime_Error_Module__loggerObj__C
800131dc   xdc_runtime_Error_Module__state__V
8000b820   xdc_runtime_Error_check__E
8000c340   xdc_runtime_Error_getSite__E
8000b860   xdc_runtime_Error_init__E
8000f3f8   xdc_runtime_Error_maxDepth__C
800055c0   xdc_runtime_Error_policyDefault__E
8000f354   xdc_runtime_Error_policyFxn__C
8000f358   xdc_runtime_Error_policy__C
80008980   xdc_runtime_Error_print__E
8000f35c   xdc_runtime_Error_raiseHook__C
8000c360   xdc_runtime_Error_raiseX__E
800099a0   xdc_runtime_Error_setX__E
8000c380   xdc_runtime_Gate_enterSystem__E
8000c3a0   xdc_runtime_Gate_leaveSystem__E
8000f360   xdc_runtime_IFilterLogger_Interface__BASE__C
8000f364   xdc_runtime_IGateProvider_Interface__BASE__C
8000f368   xdc_runtime_IHeap_Interface__BASE__C
8000f36c   xdc_runtime_ILogger_Interface__BASE__C
8000f370   xdc_runtime_IModule_Interface__BASE__C
8000f374   xdc_runtime_Log_L_error__C
8000f378   xdc_runtime_LoggerBuf_E_badLevel__C
8000b8a0   xdc_runtime_LoggerBuf_Handle__label__S
80012410   xdc_runtime_LoggerBuf_Instance_State_0_entryArr__A
8000b8e0   xdc_runtime_LoggerBuf_Instance_finalize__E
8000a240   xdc_runtime_LoggerBuf_Instance_init__E
8000c400   xdc_runtime_LoggerBuf_Module_GateProxy_enter__E
8000c420   xdc_runtime_LoggerBuf_Module_GateProxy_leave__E
8000c060   xdc_runtime_LoggerBuf_Module_GateProxy_query__E
8000eea0   xdc_runtime_LoggerBuf_Module__FXNS__C
8000f37c   xdc_runtime_LoggerBuf_Module__gateObj__C
8000f3fa   xdc_runtime_LoggerBuf_Module__id__C
800131e0   xdc_runtime_LoggerBuf_Module__root__V
800131e8   xdc_runtime_LoggerBuf_Module__state__V
8000a2c0   xdc_runtime_LoggerBuf_Module_startup__E
8000f0e0   xdc_runtime_LoggerBuf_Object__DESC__C
8000ef68   xdc_runtime_LoggerBuf_Object__PARAMS__C
8000f380   xdc_runtime_LoggerBuf_Object__count__C
80009460   xdc_runtime_LoggerBuf_Object__create__S
8000b920   xdc_runtime_LoggerBuf_Object__delete__S
8000b960   xdc_runtime_LoggerBuf_Object__get__S
800135c8   xdc_runtime_LoggerBuf_Object__table__V
8000bf00   xdc_runtime_LoggerBuf_TimestampProxy_get32__E
8000bf20   xdc_runtime_LoggerBuf_TimestampProxy_get64__E
8000bd80   xdc_runtime_LoggerBuf_TimestampProxy_getFreq__E
8000c440   xdc_runtime_LoggerBuf_disable__E
8000c460   xdc_runtime_LoggerBuf_enable__E
8000f3fc   xdc_runtime_LoggerBuf_filterByLevel__C
8000a340   xdc_runtime_LoggerBuf_filterOutEvent__I
80008320   xdc_runtime_LoggerBuf_getFilterLevel__E
8000b9a0   xdc_runtime_LoggerBuf_reset__E
80007cc0   xdc_runtime_LoggerBuf_setFilterLevel__E
8000f384   xdc_runtime_LoggerBuf_statusLogger__C
8000b9e0   xdc_runtime_LoggerBuf_write0__E
8000c480   xdc_runtime_LoggerBuf_write1__E
8000c4a0   xdc_runtime_LoggerBuf_write2__E
80005ec0   xdc_runtime_LoggerBuf_write4__E
80004180   xdc_runtime_LoggerBuf_write8__E
8000c060   xdc_runtime_Main_Module_GateProxy_query__E
8000c4c0   xdc_runtime_Memory_HeapProxy_alloc__E
8000c4e0   xdc_runtime_Memory_HeapProxy_free__E
8000f3fe   xdc_runtime_Memory_Module__id__C
800131f0   xdc_runtime_Memory_Module__state__V
80008a60   xdc_runtime_Memory_alloc__E
8000c500   xdc_runtime_Memory_calloc__E
8000f388   xdc_runtime_Memory_defaultHeapInstance__C
8000ba20   xdc_runtime_Memory_free__E
8000c520   xdc_runtime_Memory_getMaxDefaultTypeAlign__E
8000af80   xdc_runtime_Memory_valloc__E
800131f4   xdc_runtime_Registry_Module__state__V
8000ba60   xdc_runtime_Registry_findById__E
800131fc   xdc_runtime_Startup_Module__state__V
00000001   xdc_runtime_Startup__EXECFXN__C
00000001   xdc_runtime_Startup__RESETFXN__C
8000f38c   xdc_runtime_Startup_execImpl__C
80008420   xdc_runtime_Startup_exec__E
8000c540   xdc_runtime_Startup_exec__I
8000f190   xdc_runtime_Startup_firstFxns__A
8000f198   xdc_runtime_Startup_firstFxns__C
8000f1a0   xdc_runtime_Startup_lastFxns__C
8000f390   xdc_runtime_Startup_maxPasses__C
80007220   xdc_runtime_Startup_reset__I
8000c560   xdc_runtime_Startup_rtsDone__E
8000f100   xdc_runtime_Startup_sfxnRts__A
8000f394   xdc_runtime_Startup_sfxnRts__C
8000eee0   xdc_runtime_Startup_sfxnTab__A
8000f398   xdc_runtime_Startup_sfxnTab__C
800057a0   xdc_runtime_Startup_startMods__I
80012610   xdc_runtime_SysMin_Module_State_0_outbuf__A
80013204   xdc_runtime_SysMin_Module__state__V
8000afe0   xdc_runtime_SysMin_Module_startup__E
80009a40   xdc_runtime_SysMin_abort__E
8000f39c   xdc_runtime_SysMin_bufSize__C
8000b040   xdc_runtime_SysMin_exit__E
8000f400   xdc_runtime_SysMin_flushAtExit__C
80009ae0   xdc_runtime_SysMin_flush__E
8000f3a0   xdc_runtime_SysMin_outputFunc__C
8000b0a0   xdc_runtime_SysMin_output__I
80009b80   xdc_runtime_SysMin_putch__E
8000c580   xdc_runtime_SysMin_ready__E
8000c5a0   xdc_runtime_System_Module_GateProxy_enter__E
8000c5c0   xdc_runtime_System_Module_GateProxy_leave__E
8000c060   xdc_runtime_System_Module_GateProxy_query__E
80013620   xdc_runtime_System_Module_State_0_atexitHandlers__A
8000f3a4   xdc_runtime_System_Module__gateObj__C
80013210   xdc_runtime_System_Module__state__V
8000c5e0   xdc_runtime_System_Module_startup__E
80009a40   xdc_runtime_System_SupportProxy_abort__E
8000b040   xdc_runtime_System_SupportProxy_exit__E
80009ae0   xdc_runtime_System_SupportProxy_flush__E
80009b80   xdc_runtime_System_SupportProxy_putch__E
8000c580   xdc_runtime_System_SupportProxy_ready__E
8000f3a8   xdc_runtime_System_abortFxn__C
8000bcc0   xdc_runtime_System_abortStd__E
8000baa0   xdc_runtime_System_abort__E
8000bae0   xdc_runtime_System_aprintf__E
8000c600   xdc_runtime_System_aprintf_va__E
8000c600   xdc_runtime_System_aprintf_va__F
8000a3c0   xdc_runtime_System_atexit__E
8000b100   xdc_runtime_System_avprintf__E
80000000   xdc_runtime_System_doPrint__I
8000f3ac   xdc_runtime_System_exitFxn__C
80008da0   xdc_runtime_System_exitStd__E
8000bb20   xdc_runtime_System_exit__E
8000f3b0   xdc_runtime_System_extendFxn__C
80009ae0   xdc_runtime_System_flush__E
80009520   xdc_runtime_System_formatNum__I
8000f3b4   xdc_runtime_System_maxAtexitHandlers__C
80004660   xdc_runtime_System_printfExtend__I
8000bb60   xdc_runtime_System_printf__E
8000c620   xdc_runtime_System_printf_va__E
8000c620   xdc_runtime_System_printf_va__F
8000a440   xdc_runtime_System_processAtExit__E
8000a4c0   xdc_runtime_System_putchar__I
8000b160   xdc_runtime_System_vprintf__E
8000c640   xdc_runtime_System_vsnprintf__E
80013218   xdc_runtime_Text_Module__state__V
8000f402   xdc_runtime_Text_charCnt__C
8000c680   xdc_runtime_Text_charTab__A
8000f3b8   xdc_runtime_Text_charTab__C
8000b1c0   xdc_runtime_Text_cordText__E
8000f404   xdc_runtime_Text_isLoaded__C
8000f3bc   xdc_runtime_Text_nameEmpty__C
8000f3c0   xdc_runtime_Text_nameStatic__C
8000f3c4   xdc_runtime_Text_nameUnknown__C
8000ec40   xdc_runtime_Text_nodeTab__A
8000f3c8   xdc_runtime_Text_nodeTab__C
8000a540   xdc_runtime_Text_printVisFxn__I
80007de0   xdc_runtime_Text_putLab__E
80007f00   xdc_runtime_Text_putMod__E
80006080   xdc_runtime_Text_putSite__E
8000f406   xdc_runtime_Text_registryModsLastId__C
8000bba0   xdc_runtime_Text_ropeText__E
8000f408   xdc_runtime_Text_unnamedModsLastId__C
80008b40   xdc_runtime_Text_visitRope2__I
8000f3cc   xdc_runtime_Text_visitRopeFxn__C
8000c660   xdc_runtime_Text_visitRope__I
80009c20   xdc_runtime_Text_xprintf__I
8000bf00   xdc_runtime_Timestamp_SupportProxy_get32__E
8000bf20   xdc_runtime_Timestamp_SupportProxy_get64__E
8000bd80   xdc_runtime_Timestamp_SupportProxy_getFreq__E
8000bf00   xdc_runtime_Timestamp_get32__E
8000bf20   xdc_runtime_Timestamp_get64__E
8000bd80   xdc_runtime_Timestamp_getFreq__E


GLOBAL SYMBOLS: SORTED BY Symbol Address 

address    name
--------   ----
00000000   __TI_STATIC_BASE
00000000   _argsize
00000000   ti_sysbios_family_c66_Cache_l2Size
00000001   __TI_args_main
00000001   xdc_runtime_Startup__EXECFXN__C
00000001   xdc_runtime_Startup__RESETFXN__C
00002000   __TI_STACK_SIZE
00008000   ti_sysbios_family_c66_Cache_l1dSize
00008000   ti_sysbios_family_c66_Cache_l1pSize
80000000   __ASM__
80000000   xdc_runtime_System_doPrint__I
80000058   __ISA__
80000070   __PLAT__
80000098   __TARG__
800000c0   __TRDR__
80000880   ti_sysbios_family_c64p_Exception_handler__I
80001000   ti_sysbios_knl_Semaphore_pend__E
80001780   ti_sysbios_heaps_HeapMem_allocUnprotected__E
80001d60   ti_sysbios_heaps_HeapMem_freeUnprotected__E
80002300   ti_sysbios_knl_Task_Instance_finalize__E
800027a0   ti_sysbios_knl_Task_sleep__E
80002c20   ti_sysbios_timers_dmtimer_Timer_checkFreq__I
80002fc0   ti_sysbios_knl_Task_Instance_init__E
80003340   ti_sysbios_timers_dmtimer_Timer_deviceConfig__I
800036a0   ti_sysbios_heaps_HeapMem_Instance_init__E
80003980   ti_sysbios_knl_Task_Module_startup__E
80003c60   ti_sysbios_knl_Clock_workFunc__E
80003f00   ti_sysbios_knl_Semaphore_post__E
80004180   xdc_runtime_LoggerBuf_write8__E
80004400   ti_sysbios_family_c64p_Hwi_dispatchCore__I
80004660   xdc_runtime_System_printfExtend__I
800048c0   __c6xabi_divull
80004b00   ti_sysbios_family_c64p_Exception_internalHandler__I
80004d40   ti_sysbios_timers_dmtimer_Timer_setPeriodMicroSecs__E
80004f80   ti_sysbios_knl_Swi_run__I
800051a0   xdc_runtime_Core_createObject__I
800053c0   ti_sysbios_family_c64p_Hwi_dispatchAlways
800055c0   xdc_runtime_Error_policyDefault__E
800057a0   xdc_runtime_Startup_startMods__I
80005980   ti_sysbios_family_c66_Cache_block__I
80005b40   ti_sysbios_knl_Task_checkStacks__E
80005d00   ti_sysbios_knl_Task_exit__E
80005ec0   xdc_runtime_LoggerBuf_write4__E
80006080   xdc_runtime_Text_putSite__E
80006240   ti_sysbios_gates_GateMutex_enter__E
800063e0   ti_sysbios_knl_Task_schedule__I
80006700   ti_sysbios_family_c64p_Exception_dispatch__E
80006880   ti_sysbios_knl_Task_startCore__E
80006a00   xdc_runtime_Core_constructObject__I
80006b80   ti_sysbios_family_c66_Cache_getL2InitSize__I
80006ce0   ti_sysbios_knl_Swi_post__E
80006e40   ti_sysbios_timers_dmtimer_Timer_start__E
80006fa0   _auto_init_elf
800070e0   ti_sysbios_family_c64p_Hwi_Module_startup__E
80007220   ti_sysbios_family_c66_Cache_startup__I
80007220   xdc_runtime_Startup_reset__I
80007360   ti_sysbios_knl_Semaphore_Instance_init__E
800074a0   ti_sysbios_knl_Task_blockI__E
800075e0   ti_sysbios_knl_Task_postInit__I
80007720   ti_sysbios_family_c66_Cache_getL1DInitSize__I
80007840   ti_sysbios_family_c66_Cache_getL1PInitSize__I
80007960   ti_sysbios_timers_dmtimer_Timer_Module_startup__E
80007a80   ti_sysbios_timers_dmtimer_Timer_initDevice__I
80007ba0   xdc_runtime_Core_deleteObject__I
80007cc0   xdc_runtime_LoggerBuf_setFilterLevel__E
80007de0   xdc_runtime_Text_putLab__E
80007f00   xdc_runtime_Text_putMod__E
80008020   ti_sysbios_knl_Swi_restoreHwi__E
80008120   ti_sysbios_knl_Swi_schedule__I
80008220   ti_sysbios_knl_Task_unblockI__E
80008320   xdc_runtime_LoggerBuf_getFilterLevel__E
80008420   xdc_runtime_Startup_exec__E
80008520   __TI_zero_init
80008600   memset
800086e0   ti_sysbios_knl_Swi_runLoop__I
800087c0   ti_sysbios_knl_Swi_startup__E
800088a0   ti_sysbios_knl_Clock_TimerProxy_startup__E
800088a0   ti_sysbios_timers_dmtimer_Timer_startup__E
80008980   xdc_runtime_Error_print__E
80008a60   xdc_runtime_Memory_alloc__E
80008b40   xdc_runtime_Text_visitRope2__I
80008c20   HOSTwrite
80008ce0   __c6xabi_divu
80008ce0   __divu
80008da0   exit
80008da0   xdc_runtime_System_exitStd__E
80008e60   taskFxn
80008ea4   main
80008f20   ti_sysbios_heaps_HeapMem_alloc__E
80008fe0   ti_sysbios_heaps_HeapMem_getStats__E
800090a0   ti_sysbios_knl_Clock_logTick__E
80009160   ti_sysbios_knl_Task_allBlockedFunction__I
80009220   ti_sysbios_knl_Task_create
800092e0   ti_sysbios_timers_dmtimer_Timer_stop__E
800093a0   __TI_tls_init
80009460   xdc_runtime_LoggerBuf_Object__create__S
80009520   xdc_runtime_System_formatNum__I
800095e0   __c6xabi_remu
800095e0   __remu
80009680   _c_int00
80009720   memcpy
800097c0   ti_sysbios_family_c64p_Exception_Module_startup__E
80009860   ti_sysbios_heaps_HeapMem_init__I
80009900   xdc_runtime_Assert_raise__I
800099a0   xdc_runtime_Error_setX__E
80009a40   xdc_runtime_SysMin_abort__E
80009a40   xdc_runtime_System_SupportProxy_abort__E
80009ae0   xdc_runtime_SysMin_flush__E
80009ae0   xdc_runtime_System_SupportProxy_flush__E
80009ae0   xdc_runtime_System_flush__E
80009b80   xdc_runtime_SysMin_putch__E
80009b80   xdc_runtime_System_SupportProxy_putch__E
80009c20   xdc_runtime_Text_xprintf__I
80009cc0   __c6xabi_llshl
80009d40   ti_sysbios_family_c62_TaskSupport_swap__E
80009d40   ti_sysbios_knl_Task_SupportProxy_swap__E
80009dc0   readmsg
80009e40   ti_sysbios_family_c64p_Hwi_dispatchC__I
80009ec0   ti_sysbios_family_c64p_Hwi_getStackInfo__E
80009ec0   ti_sysbios_hal_Hwi_HwiProxy_getStackInfo__E
80009ec0   ti_sysbios_hal_Hwi_getStackInfo__E
80009f40   ti_sysbios_hal_Hwi_checkStack
80009fc0   ti_sysbios_hal_Hwi_initStack
8000a040   ti_sysbios_knl_Idle_run__E
8000a0c0   ti_sysbios_knl_Task_restore__E
8000a140   xdc_runtime_Core_assignLabel__I
8000a1c0   xdc_runtime_Core_assignParams__I
8000a240   xdc_runtime_LoggerBuf_Instance_init__E
8000a2c0   xdc_runtime_LoggerBuf_Module_startup__E
8000a340   xdc_runtime_LoggerBuf_filterOutEvent__I
8000a3c0   xdc_runtime_System_atexit__E
8000a440   xdc_runtime_System_processAtExit__E
8000a4c0   xdc_runtime_System_putchar__I
8000a540   xdc_runtime_Text_printVisFxn__I
8000a5c0   __c6xabi_llshru
8000a620   _subcull
8000a680   ti_sysbios_family_c64p_Hwi_switchAndDispatch__I
8000a6e0   ti_sysbios_family_xxx_Hwi_switchAndRunFunc
8000a740   ti_sysbios_BIOS_atExitFunc__I
8000a7a0   ti_sysbios_BIOS_errorRaiseHook__I
8000a800   ti_sysbios_BIOS_registerRTSLock__I
8000a860   ti_sysbios_BIOS_removeRTSLock__I
8000a8c0   ti_sysbios_BIOS_rtsUnlock__I
8000a920   ti_sysbios_BIOS_startFunc__I
8000a980   ti_sysbios_family_c62_TaskSupport_start__E
8000a980   ti_sysbios_knl_Task_SupportProxy_start__E
8000a9e0   ti_sysbios_family_c66_Cache_Module_startup__E
8000aa40   ti_sysbios_gates_GateHwi_Object__create__S
8000aaa0   ti_sysbios_gates_GateMutex_Object__create__S
8000ab00   ti_sysbios_heaps_HeapMem_Object__create__S
8000ab60   ti_sysbios_heaps_HeapMem_free__E
8000abc0   ti_sysbios_knl_Clock_Module_startup__E
8000ac20   ti_sysbios_knl_Clock_doTick__I
8000ac80   ti_sysbios_knl_Queue_construct
8000ace0   ti_sysbios_knl_Semaphore_construct
8000ad40   ti_sysbios_knl_Semaphore_pendTimeout__I
8000ada0   ti_sysbios_knl_Swi_Module_startup__E
8000ae00   ti_sysbios_knl_Task_enter__I
8000ae60   ti_sysbios_knl_Task_processVitalTaskFlag__I
8000aec0   ti_sysbios_timers_dmtimer_Timer_stub__E
8000af20   writemsg
8000af78   C$$IO$$
8000af80   xdc_runtime_Memory_valloc__E
8000afe0   xdc_runtime_SysMin_Module_startup__E
8000b040   xdc_runtime_SysMin_exit__E
8000b040   xdc_runtime_System_SupportProxy_exit__E
8000b0a0   xdc_runtime_SysMin_output__I
8000b100   xdc_runtime_System_avprintf__E
8000b160   xdc_runtime_System_vprintf__E
8000b1c0   xdc_runtime_Text_cordText__E
8000b220   __c6xabi_strasgi_64plus
8000b220   __strasgi_64plus
8000b260   _args_main
8000b2a0   ti_sysbios_family_c62_TaskSupport_buildTaskStack
8000b2e0   ti_sysbios_BIOS_exitFunc__I
8000b320   ti_sysbios_BIOS_rtsLock__I
8000b360   ti_sysbios_family_c64p_Hwi_Module__startupDone__F
8000b360   ti_sysbios_family_c64p_Hwi_Module__startupDone__S
8000b3a0   ti_sysbios_family_c64p_Hwi_disableInterrupt__E
8000b3a0   ti_sysbios_hal_Hwi_HwiProxy_disableInterrupt__E
8000b3a0   ti_sysbios_hal_Hwi_disableInterrupt__E
8000b3e0   ti_sysbios_family_c64p_Hwi_enableInterrupt__E
8000b3e0   ti_sysbios_hal_Hwi_HwiProxy_enableInterrupt__E
8000b3e0   ti_sysbios_hal_Hwi_enableInterrupt__E
8000b420   ti_sysbios_family_shared_vayu_TimerSupport_Module__startupDone__F
8000b420   ti_sysbios_family_shared_vayu_TimerSupport_Module__startupDone__S
8000b460   ti_sysbios_gates_GateHwi_Handle__label__S
8000b4a0   ti_sysbios_gates_GateHwi_Object__delete__S
8000b4e0   ti_sysbios_gates_GateMutex_Handle__label__S
8000b520   ti_sysbios_gates_GateMutex_Instance_init__E
8000b560   ti_sysbios_gates_GateMutex_Object__delete__S
8000b5a0   ti_sysbios_gates_GateMutex_leave__E
8000b5e0   ti_sysbios_heaps_HeapMem_Handle__label__S
8000b620   ti_sysbios_heaps_HeapMem_Object__delete__S
8000b660   ti_sysbios_heaps_HeapMem_Object__get__S
8000b6a0   ti_sysbios_knl_Queue_Object__destruct__S
8000b6e0   ti_sysbios_knl_Semaphore_Object__destruct__S
8000b720   ti_sysbios_knl_Swi_Object__get__S
8000b760   ti_sysbios_knl_Task_Object__get__S
8000b7a0   ti_sysbios_knl_Task_sleepTimeout__I
8000b7e0   ti_sysbios_timers_dmtimer_Timer_Module__startupDone__F
8000b7e0   ti_sysbios_timers_dmtimer_Timer_Module__startupDone__S
8000b820   xdc_runtime_Error_check__E
8000b860   xdc_runtime_Error_init__E
8000b8a0   xdc_runtime_LoggerBuf_Handle__label__S
8000b8e0   xdc_runtime_LoggerBuf_Instance_finalize__E
8000b920   xdc_runtime_LoggerBuf_Object__delete__S
8000b960   xdc_runtime_LoggerBuf_Object__get__S
8000b9a0   xdc_runtime_LoggerBuf_reset__E
8000b9e0   xdc_runtime_LoggerBuf_write0__E
8000ba20   xdc_runtime_Memory_free__E
8000ba60   xdc_runtime_Registry_findById__E
8000baa0   xdc_runtime_System_abort__E
8000bae0   xdc_runtime_System_aprintf__E
8000bb20   xdc_runtime_System_exit__E
8000bb60   xdc_runtime_System_printf__E
8000bba0   xdc_runtime_Text_ropeText__E
8000bbe0   LoggerBuf_instanceStartup
8000bc00   __xdc__init
8000bc20   _nop
8000bc40   _register_lock
8000bc60   _register_synch_api
8000bc80   _register_unlock
8000bca0   ti_sysbios_family_c62_TaskSupport_glue
8000bcc0   C$$EXIT
8000bcc0   abort
8000bcc0   xdc_runtime_System_abortStd__E
8000bce0   __TI_decompress_none
8000bd00   __TI_decompress_rle24
8000bd20   ti_sysbios_BIOS_RtsGateProxy_enter__E
8000bd40   ti_sysbios_BIOS_RtsGateProxy_leave__E
8000bd60   ti_sysbios_BIOS_exit__E
8000bd80   ti_sysbios_BIOS_getCpuFreq__E
8000bd80   ti_sysbios_family_c64p_TimestampProvider_getFreq__E
8000bd80   xdc_runtime_LoggerBuf_TimestampProxy_getFreq__E
8000bd80   xdc_runtime_Timestamp_SupportProxy_getFreq__E
8000bd80   xdc_runtime_Timestamp_getFreq__E
8000bda0   ti_sysbios_BIOS_linkedWithIncorrectBootLibrary__E
8000bdc0   ti_sysbios_BIOS_nullFunc__I
8000bde0   ti_sysbios_BIOS_setThreadType__E
8000be00   ti_sysbios_BIOS_start__E
8000be20   ti_sysbios_family_c62_TaskSupport_Module__startupDone__S
8000be40   ti_sysbios_family_c62_TaskSupport_checkStack__E
8000be40   ti_sysbios_knl_Task_SupportProxy_checkStack__E
8000be60   ti_sysbios_family_c62_TaskSupport_getStackAlignment__E
8000be60   ti_sysbios_knl_Task_SupportProxy_getStackAlignment__E
8000be80   ti_sysbios_family_c64p_Hwi_clearInterrupt__E
8000be80   ti_sysbios_hal_Hwi_HwiProxy_clearInterrupt__E
8000be80   ti_sysbios_hal_Hwi_clearInterrupt__E
8000bea0   ti_sysbios_family_c64p_Hwi_startup__E
8000bea0   ti_sysbios_hal_Hwi_HwiProxy_startup__E
8000bea0   ti_sysbios_hal_Hwi_startup__E
8000bec0   ti_sysbios_family_c64p_Hwi_switchFromBootStack__E
8000bec0   ti_sysbios_hal_Hwi_HwiProxy_switchFromBootStack__E
8000bee0   ti_sysbios_family_c64p_TimestampProvider_Module_startup__E
8000bf00   ti_sysbios_family_c64p_TimestampProvider_get32__E
8000bf00   xdc_runtime_LoggerBuf_TimestampProxy_get32__E
8000bf00   xdc_runtime_Timestamp_SupportProxy_get32__E
8000bf00   xdc_runtime_Timestamp_get32__E
8000bf20   ti_sysbios_family_c64p_TimestampProvider_get64__E
8000bf20   xdc_runtime_LoggerBuf_TimestampProxy_get64__E
8000bf20   xdc_runtime_Timestamp_SupportProxy_get64__E
8000bf20   xdc_runtime_Timestamp_get64__E
8000bf40   ti_sysbios_family_c66_Cache_RTSSynchInv__I
8000bf60   ti_sysbios_family_c66_Cache_RTSSynchWbInv__I
8000bf80   ti_sysbios_family_c66_Cache_RTSSynchWb__I
8000bfa0   ti_sysbios_family_c66_Cache_wait__E
8000bfc0   ti_sysbios_family_shared_vayu_TimerSupport_Module_startup__E
8000bfe0   ti_sysbios_family_shared_vayu_TimerSupport_enable__E
8000bfe0   ti_sysbios_timers_dmtimer_Timer_TimerSupportProxy_enable__E
8000c000   ti_sysbios_gates_GateHwi_Instance_init__E
8000c020   ti_sysbios_gates_GateHwi_enter__E
8000c040   ti_sysbios_gates_GateHwi_leave__E
8000c060   ti_sysbios_gates_GateHwi_query__E
8000c060   xdc_runtime_LoggerBuf_Module_GateProxy_query__E
8000c060   xdc_runtime_Main_Module_GateProxy_query__E
8000c060   xdc_runtime_System_Module_GateProxy_query__E
8000c080   ti_sysbios_gates_GateMutex_Instance_finalize__E
8000c0a0   ti_sysbios_BIOS_RtsGateProxy_query__E
8000c0a0   ti_sysbios_gates_GateMutex_query__E
8000c0a0   ti_sysbios_heaps_HeapMem_Module_GateProxy_query__E
8000c0c0   ti_sysbios_hal_Hwi_HwiProxy_Module__startupDone__S
8000c0e0   ti_sysbios_hal_Hwi_Module_startup__E
8000c100   ti_sysbios_heaps_HeapMem_Module_GateProxy_enter__E
8000c120   ti_sysbios_heaps_HeapMem_Module_GateProxy_leave__E
8000c140   ti_sysbios_heaps_HeapMem_isBlocking__E
8000c160   ti_sysbios_knl_Clock_TimerProxy_Module__startupDone__S
8000c180   ti_sysbios_knl_Clock_TimerProxy_getMaxTicks__E
8000c1a0   ti_sysbios_knl_Idle_loop__E
8000c1c0   ti_sysbios_knl_Queue_Instance_init__E
8000c1e0   ti_sysbios_knl_Queue_Object__get__S
8000c200   ti_sysbios_knl_Queue_destruct
8000c220   ti_sysbios_knl_Queue_empty__E
8000c240   ti_sysbios_knl_Semaphore_Instance_finalize__E
8000c260   ti_sysbios_knl_Semaphore_destruct
8000c280   ti_sysbios_knl_Swi_disable__E
8000c2a0   ti_sysbios_knl_Task_SupportProxy_Module__startupDone__S
8000c2c0   ti_sysbios_knl_Task_disable__E
8000c2e0   ti_sysbios_knl_Task_startup__E
8000c300   ti_sysbios_timers_dmtimer_Timer_TimerSupportProxy_Module__startupDone__S
8000c320   ti_sysbios_timers_dmtimer_Timer_getMaxTicks__E
8000c340   xdc_runtime_Error_getSite__E
8000c360   xdc_runtime_Error_raiseX__E
8000c380   xdc_runtime_Gate_enterSystem__E
8000c3a0   xdc_runtime_Gate_leaveSystem__E
8000c400   xdc_runtime_LoggerBuf_Module_GateProxy_enter__E
8000c420   xdc_runtime_LoggerBuf_Module_GateProxy_leave__E
8000c440   xdc_runtime_LoggerBuf_disable__E
8000c460   xdc_runtime_LoggerBuf_enable__E
8000c480   xdc_runtime_LoggerBuf_write1__E
8000c4a0   xdc_runtime_LoggerBuf_write2__E
8000c4c0   xdc_runtime_Memory_HeapProxy_alloc__E
8000c4e0   xdc_runtime_Memory_HeapProxy_free__E
8000c500   xdc_runtime_Memory_calloc__E
8000c520   xdc_runtime_Memory_getMaxDefaultTypeAlign__E
8000c540   xdc_runtime_Startup_exec__I
8000c560   xdc_runtime_Startup_rtsDone__E
8000c580   xdc_runtime_SysMin_ready__E
8000c580   xdc_runtime_System_SupportProxy_ready__E
8000c5a0   xdc_runtime_System_Module_GateProxy_enter__E
8000c5c0   xdc_runtime_System_Module_GateProxy_leave__E
8000c5e0   xdc_runtime_System_Module_startup__E
8000c600   xdc_runtime_System_aprintf_va__E
8000c600   xdc_runtime_System_aprintf_va__F
8000c620   xdc_runtime_System_printf_va__E
8000c620   xdc_runtime_System_printf_va__F
8000c640   xdc_runtime_System_vsnprintf__E
8000c660   xdc_runtime_Text_visitRope__I
8000c680   xdc_runtime_Text_charTab__A
8000e840   ti_sysbios_family_c66_Cache_marvalues__C
8000ec40   xdc_runtime_Text_nodeTab__A
8000ee64   ti_sysbios_knl_Task_Object__PARAMS__C
8000eea0   xdc_runtime_LoggerBuf_Module__FXNS__C
8000eedc   ti_sysbios_family_c62_TaskSupport_stackAlignment__C
8000eee0   xdc_runtime_Startup_sfxnTab__A
8000ef40   ti_sysbios_heaps_HeapMem_Module__FXNS__C
8000ef68   xdc_runtime_LoggerBuf_Object__PARAMS__C
8000ef90   ti_sysbios_gates_GateHwi_Module__FXNS__C
8000efb4   ti_sysbios_gates_GateMutex_Module__FXNS__C
8000efd8   ti_sysbios_heaps_HeapMem_Object__PARAMS__C
8000effc   ti_sysbios_knl_Semaphore_Object__PARAMS__C
8000f020   ti_sysbios_gates_GateHwi_Object__DESC__C
8000f040   ti_sysbios_gates_GateMutex_Object__DESC__C
8000f060   ti_sysbios_heaps_HeapMem_Object__DESC__C
8000f080   ti_sysbios_knl_Queue_Object__DESC__C
8000f0a0   ti_sysbios_knl_Semaphore_Object__DESC__C
8000f0c0   ti_sysbios_knl_Task_Object__DESC__C
8000f0e0   xdc_runtime_LoggerBuf_Object__DESC__C
8000f100   xdc_runtime_Startup_sfxnRts__A
8000f11a   ti_sysbios_family_c64p_Exception_Module__id__C
8000f11c   ti_sysbios_gates_GateHwi_Object__PARAMS__C
8000f134   ti_sysbios_gates_GateMutex_Object__PARAMS__C
8000f14c   ti_sysbios_knl_Queue_Object__PARAMS__C
8000f164   ti_sysbios_family_c64p_Exception_E_exceptionMax__C
8000f17a   ti_sysbios_family_c64p_Exception_useInternalBuffer__C
8000f184   ti_sysbios_knl_Idle_funcList__C
8000f18c   ti_sysbios_family_c64p_Exception_exceptionHook__C
8000f190   xdc_runtime_Startup_firstFxns__A
8000f198   xdc_runtime_Startup_firstFxns__C
8000f1a0   xdc_runtime_Startup_lastFxns__C
8000f1a8   ti_sysbios_family_c64p_Exception_externalHook__C
8000f1ac   ti_sysbios_family_c64p_Exception_internalHook__C
8000f1b0   ti_sysbios_family_c64p_Exception_nmiHook__C
8000f1b4   ti_sysbios_family_c64p_Hwi_LD_end__C
8000f1b8   ti_sysbios_family_c64p_Hwi_LM_begin__C
8000f1bc   ti_sysbios_family_c64p_Hwi_Module__diagsEnabled__C
8000f1c0   ti_sysbios_family_c64p_Hwi_Module__diagsIncluded__C
8000f1c4   ti_sysbios_family_c64p_Hwi_Module__diagsMask__C
8000f1c8   ti_sysbios_family_c64p_Hwi_Module__loggerFxn1__C
8000f1cc   ti_sysbios_family_c64p_Hwi_Module__loggerFxn8__C
8000f1d0   ti_sysbios_family_c64p_Hwi_Module__loggerObj__C
8000f1d4   ti_sysbios_family_c66_Cache_E_invalidL1CacheSize__C
8000f1d8   ti_sysbios_family_c66_Cache_E_invalidL2CacheSize__C
8000f1dc   ti_sysbios_family_c66_Cache_atomicBlockSize__C
8000f1e0   ti_sysbios_gates_GateMutex_A_badContext__C
8000f1e4   ti_sysbios_gates_GateMutex_Instance_State_sem__O
8000f1e8   ti_sysbios_gates_GateMutex_Module__diagsEnabled__C
8000f1ec   ti_sysbios_gates_GateMutex_Module__diagsIncluded__C
8000f1f0   ti_sysbios_gates_GateMutex_Module__diagsMask__C
8000f1f4   ti_sysbios_hal_Hwi_E_stackOverflow__C
8000f1f8   ti_sysbios_heaps_HeapMem_A_align__C
8000f1fc   ti_sysbios_heaps_HeapMem_A_heapSize__C
8000f200   ti_sysbios_heaps_HeapMem_A_invalidFree__C
8000f204   ti_sysbios_heaps_HeapMem_A_zeroBlock__C
8000f208   ti_sysbios_heaps_HeapMem_E_memory__C
8000f20c   ti_sysbios_heaps_HeapMem_Module__diagsEnabled__C
8000f210   ti_sysbios_heaps_HeapMem_Module__diagsIncluded__C
8000f214   ti_sysbios_heaps_HeapMem_Module__diagsMask__C
8000f218   ti_sysbios_heaps_HeapMem_Module__gateObj__C
8000f21c   ti_sysbios_heaps_HeapMem_Object__count__C
8000f220   ti_sysbios_heaps_HeapMem_reqAlign__C
8000f224   ti_sysbios_knl_Clock_LM_begin__C
8000f228   ti_sysbios_knl_Clock_LM_tick__C
8000f22c   ti_sysbios_knl_Clock_LW_delayed__C
8000f230   ti_sysbios_knl_Clock_Module_State_clockQ__O
8000f234   ti_sysbios_knl_Clock_Module__diagsEnabled__C
8000f238   ti_sysbios_knl_Clock_Module__diagsIncluded__C
8000f23c   ti_sysbios_knl_Clock_Module__diagsMask__C
8000f240   ti_sysbios_knl_Clock_Module__loggerFxn1__C
8000f244   ti_sysbios_knl_Clock_Module__loggerFxn2__C
8000f248   ti_sysbios_knl_Clock_Module__loggerObj__C
8000f24c   ti_sysbios_knl_Semaphore_A_badContext__C
8000f250   ti_sysbios_knl_Idle_funcList__A
8000f254   ti_sysbios_knl_Semaphore_A_noEvents__C
8000f258   ti_sysbios_knl_Semaphore_A_overflow__C
8000f25c   ti_sysbios_knl_Semaphore_A_pendTaskDisabled__C
8000f260   ti_sysbios_knl_Semaphore_Instance_State_pendQ__O
8000f264   ti_sysbios_knl_Semaphore_LM_pend__C
8000f268   ti_sysbios_knl_Semaphore_LM_post__C
8000f26c   ti_sysbios_knl_Semaphore_Module__diagsEnabled__C
8000f270   ti_sysbios_knl_Semaphore_Module__diagsIncluded__C
8000f274   ti_sysbios_knl_Semaphore_Module__diagsMask__C
8000f278   ti_sysbios_knl_Semaphore_Module__loggerFxn2__C
8000f27c   ti_sysbios_knl_Semaphore_Module__loggerFxn4__C
8000f280   ti_sysbios_knl_Semaphore_Module__loggerObj__C
8000f284   ti_sysbios_knl_Swi_LD_end__C
8000f288   ti_sysbios_knl_Swi_LM_begin__C
8000f28c   ti_sysbios_knl_Swi_LM_post__C
8000f290   ti_sysbios_knl_Swi_Module__diagsEnabled__C
8000f294   ti_sysbios_knl_Swi_Module__diagsIncluded__C
8000f298   ti_sysbios_knl_Swi_Module__diagsMask__C
8000f29c   ti_sysbios_knl_Swi_Module__loggerFxn1__C
8000f2a0   ti_sysbios_knl_Swi_Module__loggerFxn4__C
8000f2a4   ti_sysbios_knl_Swi_Module__loggerObj__C
8000f2a8   ti_sysbios_knl_Swi_Object__count__C
8000f2ac   ti_sysbios_knl_Task_A_badPriority__C
8000f2b0   ti_sysbios_knl_Task_A_badTaskState__C
8000f2b4   ti_sysbios_knl_Task_A_badThreadType__C
8000f2b8   ti_sysbios_knl_Task_A_badTimeout__C
8000f2bc   ti_sysbios_knl_Task_A_noPendElem__C
8000f2c0   ti_sysbios_knl_Task_A_sleepTaskDisabled__C
8000f2c4   ti_sysbios_knl_Task_E_spOutOfBounds__C
8000f2c8   ti_sysbios_knl_Task_E_stackOverflow__C
8000f2cc   ti_sysbios_knl_Task_LD_block__C
8000f2d0   ti_sysbios_knl_Task_LD_exit__C
8000f2d4   ti_sysbios_knl_Task_LD_ready__C
8000f2d8   ti_sysbios_knl_Task_LM_sleep__C
8000f2dc   ti_sysbios_knl_Task_LM_switch__C
8000f2e0   ti_sysbios_knl_Task_Module_State_inactiveQ__O
8000f2e4   ti_sysbios_knl_Task_Module__diagsEnabled__C
8000f2e8   ti_sysbios_knl_Task_Module__diagsIncluded__C
8000f2ec   ti_sysbios_knl_Task_Module__diagsMask__C
8000f2f0   ti_sysbios_knl_Task_Module__loggerFxn2__C
8000f2f4   ti_sysbios_knl_Task_Module__loggerFxn4__C
8000f2f8   ti_sysbios_knl_Task_Module__loggerObj__C
8000f2fc   ti_sysbios_knl_Task_Object__count__C
8000f300   ti_sysbios_knl_Task_allBlockedFunc__C
8000f304   ti_sysbios_knl_Task_defaultStackHeap__C
8000f308   ti_sysbios_knl_Task_defaultStackSize__C
8000f30c   ti_sysbios_knl_Task_numConstructedTasks__C
8000f310   ti_sysbios_timers_dmtimer_Timer_E_cannotSupport__C
8000f314   ti_sysbios_timers_dmtimer_Timer_E_freqMismatch__C
8000f318   ti_sysbios_timers_dmtimer_Timer_Module__diagsEnabled__C
8000f31c   ti_sysbios_timers_dmtimer_Timer_Module__diagsIncluded__C
8000f320   ti_sysbios_timers_dmtimer_Timer_Module__diagsMask__C
8000f324   ti_sysbios_timers_dmtimer_Timer_numTimerDevices__C
8000f328   xdc_runtime_Assert_E_assertFailed__C
8000f32c   xdc_runtime_Core_A_initializedParams__C
8000f330   xdc_runtime_Core_Module__diagsEnabled__C
8000f334   xdc_runtime_Core_Module__diagsIncluded__C
8000f338   xdc_runtime_Core_Module__diagsMask__C
8000f33c   xdc_runtime_Error_E_memory__C
8000f340   xdc_runtime_Error_Module__diagsEnabled__C
8000f344   xdc_runtime_Error_Module__diagsIncluded__C
8000f348   xdc_runtime_Error_Module__diagsMask__C
8000f34c   xdc_runtime_Error_Module__loggerFxn8__C
8000f350   xdc_runtime_Error_Module__loggerObj__C
8000f354   xdc_runtime_Error_policyFxn__C
8000f358   xdc_runtime_Error_policy__C
8000f35c   xdc_runtime_Error_raiseHook__C
8000f360   xdc_runtime_IFilterLogger_Interface__BASE__C
8000f364   xdc_runtime_IGateProvider_Interface__BASE__C
8000f368   xdc_runtime_IHeap_Interface__BASE__C
8000f36c   xdc_runtime_ILogger_Interface__BASE__C
8000f370   xdc_runtime_IModule_Interface__BASE__C
8000f374   xdc_runtime_Log_L_error__C
8000f378   xdc_runtime_LoggerBuf_E_badLevel__C
8000f37c   xdc_runtime_LoggerBuf_Module__gateObj__C
8000f380   xdc_runtime_LoggerBuf_Object__count__C
8000f384   xdc_runtime_LoggerBuf_statusLogger__C
8000f388   xdc_runtime_Memory_defaultHeapInstance__C
8000f38c   xdc_runtime_Startup_execImpl__C
8000f390   xdc_runtime_Startup_maxPasses__C
8000f394   xdc_runtime_Startup_sfxnRts__C
8000f398   xdc_runtime_Startup_sfxnTab__C
8000f39c   xdc_runtime_SysMin_bufSize__C
8000f3a0   xdc_runtime_SysMin_outputFunc__C
8000f3a4   xdc_runtime_System_Module__gateObj__C
8000f3a8   xdc_runtime_System_abortFxn__C
8000f3ac   xdc_runtime_System_exitFxn__C
8000f3b0   xdc_runtime_System_extendFxn__C
8000f3b4   xdc_runtime_System_maxAtexitHandlers__C
8000f3b8   xdc_runtime_Text_charTab__C
8000f3bc   xdc_runtime_Text_nameEmpty__C
8000f3c0   xdc_runtime_Text_nameStatic__C
8000f3c4   xdc_runtime_Text_nameUnknown__C
8000f3c8   xdc_runtime_Text_nodeTab__C
8000f3cc   xdc_runtime_Text_visitRopeFxn__C
8000f3d0   ti_sysbios_family_c64p_Hwi_Module__id__C
8000f3d2   ti_sysbios_family_c64p_Hwi_Module__loggerDefined__C
8000f3d4   ti_sysbios_family_c66_Cache_Module__id__C
8000f3d6   ti_sysbios_family_c66_Cache_registerRTSSynch__C
8000f3d8   ti_sysbios_gates_GateMutex_Module__id__C
8000f3da   ti_sysbios_hal_Hwi_Module__id__C
8000f3dc   ti_sysbios_heaps_HeapMem_Module__id__C
8000f3de   ti_sysbios_knl_Clock_Module__id__C
8000f3e0   ti_sysbios_knl_Clock_Module__loggerDefined__C
8000f3e2   ti_sysbios_knl_Semaphore_Module__id__C
8000f3e4   ti_sysbios_knl_Semaphore_Module__loggerDefined__C
8000f3e6   ti_sysbios_knl_Swi_Module__id__C
8000f3e8   ti_sysbios_knl_Swi_Module__loggerDefined__C
8000f3ea   ti_sysbios_knl_Task_Module__id__C
8000f3ec   ti_sysbios_knl_Task_Module__loggerDefined__C
8000f3ee   ti_sysbios_timers_dmtimer_Timer_Module__id__C
8000f3f0   ti_sysbios_timers_dmtimer_Timer_checkFrequency__C
8000f3f2   ti_sysbios_timers_dmtimer_Timer_startupNeeded__C
8000f3f4   xdc_runtime_Core_Module__id__C
8000f3f6   xdc_runtime_Error_Module__loggerDefined__C
8000f3f8   xdc_runtime_Error_maxDepth__C
8000f3fa   xdc_runtime_LoggerBuf_Module__id__C
8000f3fc   xdc_runtime_LoggerBuf_filterByLevel__C
8000f3fe   xdc_runtime_Memory_Module__id__C
8000f400   xdc_runtime_SysMin_flushAtExit__C
8000f402   xdc_runtime_Text_charCnt__C
8000f404   xdc_runtime_Text_isLoaded__C
8000f406   xdc_runtime_Text_registryModsLastId__C
8000f408   xdc_runtime_Text_unnamedModsLastId__C
8000f410   _stack
80011410   __TI_STACK_END
80011410   ti_sysbios_heaps_HeapMem_Instance_State_0_buf__A
80012410   xdc_runtime_LoggerBuf_Instance_State_0_entryArr__A
80012610   xdc_runtime_SysMin_Module_State_0_outbuf__A
80012810   ti_sysbios_knl_Task_Instance_State_0_stack__A
80013018   ti_sysbios_BIOS_Module__state__V
8001303c   ti_sysbios_family_c64p_Exception_Module__state__V
8001306c   ti_sysbios_family_c64p_Hwi_Module__root__V
80013074   ti_sysbios_family_c64p_Hwi_Module__state__V
800130e0   ti_sysbios_gates_GateHwi_Module__root__V
800130e8   ti_sysbios_gates_GateMutex_Module__root__V
800130f0   ti_sysbios_hal_Hwi_Module__root__V
800130f8   ti_sysbios_heaps_HeapMem_Module__root__V
80013100   ti_sysbios_knl_Clock_Module__root__V
80013108   ti_sysbios_knl_Clock_Module__state__V
80013134   ti_sysbios_knl_Queue_Module__root__V
8001313c   ti_sysbios_knl_Semaphore_Module__root__V
80013144   ti_sysbios_knl_Swi_Module__root__V
8001314c   ti_sysbios_knl_Swi_Module__state__V
80013168   ti_sysbios_knl_Task_Module__root__V
80013170   ti_sysbios_knl_Task_Module__state__V
800131b4   ti_sysbios_rts_ti_ThreadLocalStorage_Module__state__V
800131c0   ti_sysbios_timers_dmtimer_Timer_Module__root__V
800131c8   ti_sysbios_timers_dmtimer_Timer_Module__state__V
800131dc   xdc_runtime_Error_Module__state__V
800131e0   xdc_runtime_LoggerBuf_Module__root__V
800131e8   xdc_runtime_LoggerBuf_Module__state__V
800131f0   xdc_runtime_Memory_Module__state__V
800131f4   xdc_runtime_Registry_Module__state__V
800131fc   xdc_runtime_Startup_Module__state__V
80013204   xdc_runtime_SysMin_Module__state__V
80013210   xdc_runtime_System_Module__state__V
80013218   xdc_runtime_Text_Module__state__V
80013220   __xdc__init__addr
80013228   ti_sysbios_timers_dmtimer_Timer_Module_State_0_device__A
800132e8   ti_sysbios_knl_Swi_Module_State_0_readyQ__A
80013368   ti_sysbios_knl_Task_Module_State_0_readyQ__A
800133e8   ti_sysbios_timers_dmtimer_Timer_Module_State_0_intFreqs__A
80013468   ti_sysbios_timers_dmtimer_Timer_Object__table__V
800134c8   ti_sysbios_knl_Task_Object__table__V
80013518   ti_sysbios_gates_GateMutex_Object__table__V
80013558   ti_sysbios_timers_dmtimer_Timer_Module_State_0_handles__A
80013598   ti_sysbios_knl_Swi_Object__table__V
800135c8   xdc_runtime_LoggerBuf_Object__table__V
800135f0   ti_sysbios_family_c64p_Hwi_Object__table__V
80013608   ti_sysbios_heaps_HeapMem_Object__table__V
80013620   xdc_runtime_System_Module_State_0_atexitHandlers__A
80013630   _cleanup_ptr
80013634   _dtors_ptr
80013638   __TI_enable_exit_profile_output
8001363c   _lock
80013640   _unlock
80013648   ti_sysbios_hal_Hwi_Object__table__V
80013650   ti_sysbios_gates_GateHwi_Object__table__V
80013658   ti_sysbios_knl_Task_Module_State_0_idleTask__A
80013660   __CIOBUF_
80013800   ti_sysbios_family_c64p_Hwi0
80013800   ti_sysbios_family_c64p_Hwi_int0
80013820   ti_sysbios_family_c64p_Hwi_int1
80013840   ti_sysbios_family_c64p_Hwi_int2
80013860   ti_sysbios_family_c64p_Hwi_int3
80013880   ti_sysbios_family_c64p_Hwi_int4
800138a0   ti_sysbios_family_c64p_Hwi_int5
800138c0   ti_sysbios_family_c64p_Hwi_int6
800138e0   ti_sysbios_family_c64p_Hwi_int7
80013900   ti_sysbios_family_c64p_Hwi_int8
80013920   ti_sysbios_family_c64p_Hwi_int9
80013940   ti_sysbios_family_c64p_Hwi_int10
80013960   ti_sysbios_family_c64p_Hwi_int11
80013980   ti_sysbios_family_c64p_Hwi_int12
800139a0   ti_sysbios_family_c64p_Hwi_int13
800139c0   ti_sysbios_family_c64p_Hwi_int14
800139e0   ti_sysbios_family_c64p_Hwi_int15
80013e48   __TI_Handler_Table_Base
80013e54   __TI_Handler_Table_Limit
80013e60   __TI_CINIT_Base
80013e70   __TI_CINIT_Limit
ffffffff   __TI_pprof_out_hndl
ffffffff   __TI_prof_data_size
ffffffff   __TI_prof_data_start
ffffffff   __binit__
ffffffff   __c_args__
ffffffff   binit
UNDEFED    __TI_INITARRAY_Base
UNDEFED    __TI_INITARRAY_Limit
UNDEFED    __TI_TLS_INIT_Base
UNDEFED    __TI_TLS_INIT_Limit

[615 symbols]
